 Proclist

 Timestamp is 51e6ece3 (Wed Jul 17 23:13:39 2013)

 Preferred load address is 10000000

 Start         Length     Name                   Class
 0001:00000000 0000016cH .idata$5                CODE
 0001:00000170 00001b54H .rdata                  CODE
 0001:00001cd0 0000a304H .text                   CODE
 0001:0000bfd4 0000008cH .idata$2                CODE
 0001:0000c060 00000014H .idata$3                CODE
 0001:0000c074 0000016cH .idata$4                CODE
 0001:0000c1e0 0000060eH .idata$6                CODE
 0001:0000c7f0 00000192H .edata                  CODE
 0002:00000000 000001c0H .data                   DATA
 0002:000001c0 00024fe8H .bss                    DATA
 0003:00000000 00000058H .rsrc$01                DATA
 0003:00000060 00000378H .rsrc$02                DATA

  Address         Publics by Value              Rva+Base       Lib:Object

 0000:00000000       ___safe_se_handler_count   00000000     <absolute>
 0000:00000000       ___safe_se_handler_table   00000000     <absolute>
 0001:00000000       __imp__GetUserNameW@8      10001000     advapi32:ADVAPI32.dll
 0001:00000004       __imp__RegCloseKey@4       10001004     advapi32:ADVAPI32.dll
 0001:00000008       __imp__RegQueryValueExW@24 10001008     advapi32:ADVAPI32.dll
 0001:0000000c       __imp__RegConnectRegistryW@12 1000100c     advapi32:ADVAPI32.dll
 0001:00000010       __imp__SetThreadToken@8    10001010     advapi32:ADVAPI32.dll
 0001:00000014       __imp__OpenThreadToken@16  10001014     advapi32:ADVAPI32.dll
 0001:00000018       __imp__AdjustTokenPrivileges@24 10001018     advapi32:ADVAPI32.dll
 0001:0000001c       __imp__LookupPrivilegeValueW@12 1000101c     advapi32:ADVAPI32.dll
 0001:00000020       __imp__DuplicateTokenEx@24 10001020     advapi32:ADVAPI32.dll
 0001:00000024       __imp__OpenProcessToken@12 10001024     advapi32:ADVAPI32.dll
 0001:00000028       __imp__RegOpenKeyExW@20    10001028     advapi32:ADVAPI32.dll
 0001:0000002c       \177ADVAPI32_NULL_THUNK_DATA 1000102c     advapi32:ADVAPI32.dll
 0001:00000030       __imp__SetLastError@4      10001030     kernel32:KERNEL32.dll
 0001:00000034       __imp__VirtualFree@12      10001034     kernel32:KERNEL32.dll
 0001:00000038       __imp__VirtualAlloc@16     10001038     kernel32:KERNEL32.dll
 0001:0000003c       __imp__SetEvent@4          1000103c     kernel32:KERNEL32.dll
 0001:00000040       __imp__lstrcatW@8          10001040     kernel32:KERNEL32.dll
 0001:00000044       __imp__lstrcpyW@8          10001044     kernel32:KERNEL32.dll
 0001:00000048       __imp__FileTimeToSystemTime@8 10001048     kernel32:KERNEL32.dll
 0001:0000004c       __imp__lstrcmpiW@8         1000104c     kernel32:KERNEL32.dll
 0001:00000050       __imp__GetCurrentThreadId@0 10001050     kernel32:KERNEL32.dll
 0001:00000054       __imp__GetTickCount@0      10001054     kernel32:KERNEL32.dll
 0001:00000058       __imp__SystemTimeToTzSpecificLocalTime@12 10001058     kernel32:KERNEL32.dll
 0001:0000005c       __imp__GetLocalTime@4      1000105c     kernel32:KERNEL32.dll
 0001:00000060       __imp__GetSystemTimeAsFileTime@4 10001060     kernel32:KERNEL32.dll
 0001:00000064       __imp__CreateFileW@28      10001064     kernel32:KERNEL32.dll
 0001:00000068       __imp__SetPriorityClass@8  10001068     kernel32:KERNEL32.dll
 0001:0000006c       __imp__GetPriorityClass@4  1000106c     kernel32:KERNEL32.dll
 0001:00000070       __imp__lstrcmpW@8          10001070     kernel32:KERNEL32.dll
 0001:00000074       __imp__ResetEvent@4        10001074     kernel32:KERNEL32.dll
 0001:00000078       __imp__GetProcessTimes@20  10001078     kernel32:KERNEL32.dll
 0001:0000007c       __imp__GetCurrentProcessId@0 1000107c     kernel32:KERNEL32.dll
 0001:00000080       __imp__CreateEventW@16     10001080     kernel32:KERNEL32.dll
 0001:00000084       __imp__CreateMutexW@12     10001084     kernel32:KERNEL32.dll
 0001:00000088       __imp__ReadProcessMemory@20 10001088     kernel32:KERNEL32.dll
 0001:0000008c       __imp__GetLastError@0      1000108c     kernel32:KERNEL32.dll
 0001:00000090       __imp__GetCurrentThread@0  10001090     kernel32:KERNEL32.dll
 0001:00000094       __imp__OpenProcess@12      10001094     kernel32:KERNEL32.dll
 0001:00000098       __imp__TerminateProcess@8  10001098     kernel32:KERNEL32.dll
 0001:0000009c       __imp__GetDateFormatW@24   1000109c     kernel32:KERNEL32.dll
 0001:000000a0       __imp__GetTimeFormatW@24   100010a0     kernel32:KERNEL32.dll
 0001:000000a4       __imp__FileTimeToLocalFileTime@8 100010a4     kernel32:KERNEL32.dll
 0001:000000a8       __imp__LocalFree@4         100010a8     kernel32:KERNEL32.dll
 0001:000000ac       __imp__FormatMessageW@28   100010ac     kernel32:KERNEL32.dll
 0001:000000b0       __imp__GetModuleHandleW@4  100010b0     kernel32:KERNEL32.dll
 0001:000000b4       __imp__DisableThreadLibraryCalls@4 100010b4     kernel32:KERNEL32.dll
 0001:000000b8       __imp__GetProcAddress@8    100010b8     kernel32:KERNEL32.dll
 0001:000000bc       __imp__HeapFree@12         100010bc     kernel32:KERNEL32.dll
 0001:000000c0       __imp__GetProcessHeap@0    100010c0     kernel32:KERNEL32.dll
 0001:000000c4       __imp__HeapAlloc@12        100010c4     kernel32:KERNEL32.dll
 0001:000000c8       __imp__GetCurrentProcess@0 100010c8     kernel32:KERNEL32.dll
 0001:000000cc       __imp__DuplicateHandle@28  100010cc     kernel32:KERNEL32.dll
 0001:000000d0       __imp__lstrlenW@4          100010d0     kernel32:KERNEL32.dll
 0001:000000d4       __imp__lstrcpynW@12        100010d4     kernel32:KERNEL32.dll
 0001:000000d8       __imp__CreateThread@24     100010d8     kernel32:KERNEL32.dll
 0001:000000dc       __imp__TerminateThread@8   100010dc     kernel32:KERNEL32.dll
 0001:000000e0       __imp__CloseHandle@4       100010e0     kernel32:KERNEL32.dll
 0001:000000e4       __imp__Sleep@4             100010e4     kernel32:KERNEL32.dll
 0001:000000e8       __imp__ReleaseMutex@4      100010e8     kernel32:KERNEL32.dll
 0001:000000ec       __imp__WaitForSingleObject@8 100010ec     kernel32:KERNEL32.dll
 0001:000000f0       __imp__WaitForMultipleObjects@16 100010f0     kernel32:KERNEL32.dll
 0001:000000f4       __imp__WriteFile@20        100010f4     kernel32:KERNEL32.dll
 0001:000000f8       \177KERNEL32_NULL_THUNK_DATA 100010f8     kernel32:KERNEL32.dll
 0001:000000fc       __imp__WNetAddConnection2W@16 100010fc     mpr:MPR.dll
 0001:00000100       __imp__WNetCancelConnection2W@12 10001100     mpr:MPR.dll
 0001:00000104       \177MPR_NULL_THUNK_DATA    10001104     mpr:MPR.dll
 0001:00000108       __imp__SysAllocString@4    10001108     oleaut32:OLEAUT32.dll
 0001:0000010c       __imp__SysFreeString@4     1000110c     oleaut32:OLEAUT32.dll
 0001:00000110       __imp__VariantClear@4      10001110     oleaut32:OLEAUT32.dll
 0001:00000114       \177OLEAUT32_NULL_THUNK_DATA 10001114     oleaut32:OLEAUT32.dll
 0001:00000118       __imp__GetWindowThreadProcessId@8 10001118     user32:USER32.dll
 0001:0000011c       __imp__GetParent@4         1000111c     user32:USER32.dll
 0001:00000120       __imp__IsWindowVisible@4   10001120     user32:USER32.dll
 0001:00000124       __imp__GetWindowTextW@12   10001124     user32:USER32.dll
 0001:00000128       __imp__GetWindowLongW@8    10001128     user32:USER32.dll
 0001:0000012c       __imp__wsprintfW           1000112c     user32:USER32.dll
 0001:00000130       __imp__EnumWindows@8       10001130     user32:USER32.dll
 0001:00000134       __imp__ShowWindowAsync@8   10001134     user32:USER32.dll
 0001:00000138       __imp__GetWindowPlacement@8 10001138     user32:USER32.dll
 0001:0000013c       __imp__SetForegroundWindow@4 1000113c     user32:USER32.dll
 0001:00000140       __imp__SystemParametersInfoW@16 10001140     user32:USER32.dll
 0001:00000144       __imp__IsIconic@4          10001144     user32:USER32.dll
 0001:00000148       \177USER32_NULL_THUNK_DATA 10001148     user32:USER32.dll
 0001:0000014c       __imp__GetFileVersionInfoW@16 1000114c     version:VERSION.dll
 0001:00000150       __imp__GetFileVersionInfoSizeW@8 10001150     version:VERSION.dll
 0001:00000154       __imp__VerQueryValueW@16   10001154     version:VERSION.dll
 0001:00000158       \177VERSION_NULL_THUNK_DATA 10001158     version:VERSION.dll
 0001:0000015c       __imp__CoCreateInstance@20 1000115c     ole32:ole32.dll
 0001:00000160       __imp__CoUninitialize@0    10001160     ole32:ole32.dll
 0001:00000164       __imp__CoInitialize@4      10001164     ole32:ole32.dll
 0001:00000168       \177ole32_NULL_THUNK_DATA  10001168     ole32:ole32.dll
 0001:00000170       ??_C@_1BA@KLFBJALL@?$AAW?$AAm?$AAi?$AAG?$AAu?$AAi?$AAd?$AA?$AA@ 10001170     handles.obj
 0001:00000180       ??_C@_19DDLLJDOO@?$AAF?$AAi?$AAl?$AAe?$AA?$AA@ 10001180     handles.obj
 0001:0000018c       ??_C@_1BK@HCMNLOAL@?$AAI?$AAo?$AAC?$AAo?$AAm?$AAp?$AAl?$AAe?$AAt?$AAi?$AAo?$AAn?$AA?$AA@ 1000118c     handles.obj
 0001:000001a8       ??_C@_17EKANHMLE@?$AAJ?$AAo?$AAb?$AA?$AA@ 100011a8     handles.obj
 0001:000001b0       ??_C@_1BK@GACLFIOK@?$AAW?$AAa?$AAi?$AAt?$AAa?$AAb?$AAl?$AAe?$AAP?$AAo?$AAr?$AAt?$AA?$AA@ 100011b0     handles.obj
 0001:000001cc       ??_C@_19OBNDINH@?$AAP?$AAo?$AAr?$AAt?$AA?$AA@ 100011cc     handles.obj
 0001:000001d8       ??_C@_17KACEIPNC@?$AAK?$AAe?$AAy?$AA?$AA@ 100011d8     handles.obj
 0001:000001e0       ??_C@_1BA@LHDKDEEN@?$AAS?$AAe?$AAc?$AAt?$AAi?$AAo?$AAn?$AA?$AA@ 100011e0     handles.obj
 0001:000001f0       ??_C@_1BA@CBCBMBGJ@?$AAD?$AAe?$AAs?$AAk?$AAt?$AAo?$AAp?$AA?$AA@ 100011f0     handles.obj
 0001:00000200       ??_C@_1BM@JIPCCEDL@?$AAW?$AAi?$AAn?$AAd?$AAo?$AAw?$AAS?$AAt?$AAa?$AAt?$AAi?$AAo?$AAn?$AA?$AA@ 10001200     handles.obj
 0001:0000021c       ??_C@_1BA@OKEJPPOI@?$AAP?$AAr?$AAo?$AAf?$AAi?$AAl?$AAe?$AA?$AA@ 1000121c     handles.obj
 0001:0000022c       ??_C@_1M@EEEEDEMN@?$AAT?$AAi?$AAm?$AAe?$AAr?$AA?$AA@ 1000122c     handles.obj
 0001:00000238       ??_C@_1BE@NPGPGCB@?$AAS?$AAe?$AAm?$AAa?$AAp?$AAh?$AAo?$AAr?$AAe?$AA?$AA@ 10001238     handles.obj
 0001:0000024c       ??_C@_1O@FBKOCLFA@?$AAM?$AAu?$AAt?$AAa?$AAn?$AAt?$AA?$AA@ 1000124c     handles.obj
 0001:0000025c       ??_C@_1BE@EBMGBMON@?$AAE?$AAv?$AAe?$AAn?$AAt?$AAP?$AAa?$AAi?$AAr?$AA?$AA@ 1000125c     handles.obj
 0001:00000270       ??_C@_1M@JJBFPLJB@?$AAE?$AAv?$AAe?$AAn?$AAt?$AA?$AA@ 10001270     handles.obj
 0001:0000027c       ??_C@_1O@CDOGJPJJ@?$AAT?$AAh?$AAr?$AAe?$AAa?$AAd?$AA?$AA@ 1000127c     handles.obj
 0001:0000028c       ??_C@_1BA@NMDNJJOO@?$AAP?$AAr?$AAo?$AAc?$AAe?$AAs?$AAs?$AA?$AA@ 1000128c     handles.obj
 0001:0000029c       ??_C@_1M@JFPKKFCK@?$AAT?$AAo?$AAk?$AAe?$AAn?$AA?$AA@ 1000129c     handles.obj
 0001:000002a8       ??_C@_1BK@KDPOKCA@?$AAS?$AAy?$AAm?$AAb?$AAo?$AAl?$AAi?$AAc?$AAL?$AAi?$AAn?$AAk?$AA?$AA@ 100012a8     handles.obj
 0001:000002c4       ??_C@_1BE@DNDHOCGP@?$AAD?$AAi?$AAr?$AAe?$AAc?$AAt?$AAo?$AAr?$AAy?$AA?$AA@ 100012c4     handles.obj
 0001:000002d8       ??_C@_11LOCGONAA@?$AA?$AA@ 100012d8     handles.obj
 0001:0000033c       ??_C@_17CNPHIMPH@?$AA?$CF?$AAl?$AAs?$AA?$AA@ 1000133c     handles.obj
 0001:00000344       ??_C@_1BA@FDFONNEJ@?$AA?$CF?$AAs?$AA?5?$AA?$CI?$AA?$CF?$AAd?$AA?$CJ?$AA?$AA@ 10001344     handles.obj
 0001:00000354       ??_C@_1BE@ELICABCK@?$AA?$DM?$AAu?$AAn?$AAk?$AAn?$AAo?$AAw?$AAn?$AA?$DO?$AA?$AA@ 10001354     handles.obj
 0001:00000368       ??_C@_1BA@LGCEDAAB@?$AAT?$AAI?$AAD?$AA?3?$AA?5?$AA?$CF?$AAd?$AA?$AA@ 10001368     handles.obj
 0001:00000378       ??_C@_15GANGMFKL@?$AA?$CF?$AAs?$AA?$AA@ 10001378     handles.obj
 0001:00000380       ??_C@_19PEALEEJB@?$AAH?$AAK?$AAL?$AAM?$AA?$AA@ 10001380     handles.obj
 0001:0000038c       ??_C@_1BA@INBMCOAP@?$AAM?$AAA?$AAC?$AAH?$AAI?$AAN?$AAE?$AA?$AA@ 1000138c     handles.obj
 0001:0000039c       ??_C@_19NCHLBIN@?$AAH?$AAK?$AAC?$AAR?$AA?$AA@ 1000139c     handles.obj
 0001:000003a8       ??_C@_1DC@OIDKFHBF@?$AAM?$AAA?$AAC?$AAH?$AAI?$AAN?$AAE?$AA?2?$AAS?$AAO?$AAF?$AAT?$AAW?$AAA?$AAR?$AAE?$AA?2?$AAC?$AAL?$AAA?$AAS?$AAS?$AAE?$AAS?$AA?$AA@ 100013a8     handles.obj
 0001:000003dc       ??_C@_17PJOJPMPB@?$AAH?$AAK?$AAU?$AA?$AA@ 100013dc     handles.obj
 0001:000003e4       ??_C@_1BK@OEABCBLA@?$AAH?$AAK?$AAC?$AAU?$AA?2?$AAC?$AAl?$AAa?$AAs?$AAs?$AAe?$AAs?$AA?$AA@ 100013e4     handles.obj
 0001:00000400       ??_C@_19JAPAIJDE@?$AAH?$AAK?$AAC?$AAU?$AA?$AA@ 10001400     handles.obj
 0001:0000040c       ??_C@_1BC@PGMOPNLK@?$AA_?$AAC?$AAl?$AAa?$AAs?$AAs?$AAe?$AAs?$AA?$AA@ 1000140c     handles.obj
 0001:00000420       ??_C@_19KGHAHCFG@?$AAU?$AAS?$AAE?$AAR?$AA?$AA@ 10001420     handles.obj
 0001:0000042c       ??_C@_1BG@OKCBELMP@?$AA?2?$AAR?$AAE?$AAG?$AAI?$AAS?$AAT?$AAR?$AAY?$AA?2?$AA?$AA@ 1000142c     handles.obj
 0001:00000444       ??_C@_1O@EAOKCHFC@?$AA?$CF?$AA?9?$AA1?$AA3?$AAs?$AA?5?$AA?$AA@ 10001444     handles.obj
 0001:00000454       ??_C@_19DEJHOMFE@?$AA?9?$AA?$CF?$AAl?$AAu?$AA?$AA@ 10001454     handles.obj
 0001:00000460       ??_C@_1EC@MPDKEHCN@?$AA0?$AAx?$AA?$CF?$AA0?$AA2?$AAh?$AAx?$AA?$CF?$AA0?$AA2?$AAh?$AAx?$AA?$CF?$AA0?$AA2?$AAh?$AAx?$AA?$CF?$AA0?$AA2?$AAh?$AAx?$AA?$CF?$AA0?$AA2?$AAh?$AAx?$AA?$CF?$AA0?$AA2?$AAh?$AAx@ 10001460     handles.obj
 0001:000004a4       ??_C@_17IJMNDCL@?$AA?$CF?$AAl?$AAu?$AA?$AA@ 100014a4     handles.obj
 0001:000004ac       ??_C@_1BA@IGEMANKH@?$AA?2?$AAS?$AA?9?$AA?$CF?$AAl?$AAu?$AA?9?$AA?$AA@ 100014ac     handles.obj
 0001:000004bc       ??_C@_1BG@OCPCMCEA@?$AA?$CF?$AA5?$AAX?$AA?5?$AA?5?$AA?$CF?$AA0?$AA8?$AAX?$AA?5?$AA?$AA@ 100014bc     handles.obj
 0001:000004d4       ??_C@_1O@HAOIKAHJ@?$AA?$CF?$AAs?$AA?6?$AA?$CF?$AAs?$AA?6?$AA?$AA@ 100014d4     handles.obj
 0001:000004e4       ??_C@_1CK@CLFOOHFA@?$AAE?$AAx?$AAp?$AAo?$AAr?$AAt?$AAH?$AAa?$AAn?$AAd?$AAl?$AAe?$AAs?$AAU?$AAn?$AAn?$AAa?$AAm?$AAe?$AAd?$AA?$AA@ 100014e4     PCFG.OBJ
 0001:00000510       ??_C@_1BM@KMCHODLM@?$AAE?$AAx?$AAp?$AAo?$AAr?$AAt?$AAH?$AAa?$AAn?$AAd?$AAl?$AAe?$AAs?$AA?$AA@ 10001510     PCFG.OBJ
 0001:0000052c       ??_C@_1CE@GNMOKOAL@?$AAE?$AAx?$AAp?$AAo?$AAr?$AAt?$AAP?$AAe?$AAr?$AAf?$AAo?$AAr?$AAm?$AAa?$AAn?$AAc?$AAe?$AA?$AA@ 1000152c     PCFG.OBJ
 0001:00000550       ??_C@_1CI@OFLGHPDG@?$AAE?$AAx?$AAp?$AAo?$AAr?$AAt?$AAM?$AAo?$AAd?$AAu?$AAl?$AAe?$AAV?$AAe?$AAr?$AAs?$AAi?$AAo?$AAn?$AA?$AA@ 10001550     PCFG.OBJ
 0001:00000578       ??_C@_1CC@OABICAMP@?$AAE?$AAx?$AAp?$AAo?$AAr?$AAt?$AAM?$AAo?$AAd?$AAu?$AAl?$AAe?$AAI?$AAn?$AAf?$AAo?$AA?$AA@ 10001578     PCFG.OBJ
 0001:0000059c       ??_C@_1CE@JIPJNDMD@?$AAE?$AAx?$AAp?$AAo?$AAr?$AAt?$AAE?$AAn?$AAv?$AAi?$AAr?$AAo?$AAn?$AAm?$AAe?$AAn?$AAt?$AA?$AA@ 1000159c     PCFG.OBJ
 0001:000005c0       ??_C@_1CC@PNNAOHJC@?$AAA?$AAd?$AAd?$AAT?$AAo?$AAP?$AAl?$AAu?$AAg?$AAi?$AAn?$AAs?$AAM?$AAe?$AAn?$AAu?$AA?$AA@ 100015c0     PCFG.OBJ
 0001:000005e4       ??_C@_1BO@NGDOFANC@?$AAA?$AAd?$AAd?$AAT?$AAo?$AAD?$AAi?$AAs?$AAk?$AAs?$AAM?$AAe?$AAn?$AAu?$AA?$AA@ 100015e4     PCFG.OBJ
 0001:00000604       ??_C@_1BE@PKILIDFH@?$AAE?$AAn?$AAa?$AAb?$AAl?$AAe?$AAW?$AAM?$AAI?$AA?$AA@ 10001604     PCFG.OBJ
 0001:00000618       ??_7?$DialogBuilderBase@UFarDialogItem@@@@6B@ 10001618     PCFG.OBJ
 0001:00000638       ??_7PluginDialogBuilder@@6B@ 10001638     PCFG.OBJ
 0001:00000658       ??_7?$DialogItemBinding@UFarDialogItem@@@@6B@ 10001658     PCFG.OBJ
 0001:00000660       ??_7PluginCheckBoxBinding@@6B@ 10001660     PCFG.OBJ
 0001:00000668       ??_7PluginRadioButtonBinding@@6B@ 10001668     PCFG.OBJ
 0001:00000670       ??_C@_15EFLNJKHH@?$AA?$CF?$AAu?$AA?$AA@ 10001670     PCFG.OBJ
 0001:00000678       ??_7PluginIntEditFieldBinding@@6B@ 10001678     PCFG.OBJ
 0001:00000680       ??_C@_1O@BJPKKLLM@?$AAC?$AAo?$AAn?$AAf?$AAi?$AAg?$AA?$AA@ 10001680     PCFG.OBJ
 0001:00000690       ??_C@_13LHMFKAAD@?$AAM?$AA?$AA@ 10001690     Pclass.obj
 0001:00000694       ??_C@_13JCKOPPNP@?$AAK?$AA?$AA@ 10001694     Pclass.obj
 0001:00000698       ??_C@_1CC@EBBNDNOD@?$AAF?$AAu?$AAl?$AAl?$AAS?$AAc?$AAr?$AAe?$AAe?$AAn?$AAR?$AAe?$AAm?$AAo?$AAt?$AAe?$AA?$AA@ 10001698     Pclass.obj
 0001:000006bc       ??_C@_1CA@HLBJOHGN@?$AAF?$AAu?$AAl?$AAl?$AAS?$AAc?$AAr?$AAe?$AAe?$AAn?$AAL?$AAo?$AAc?$AAa?$AAl?$AA?$AA@ 100016bc     Pclass.obj
 0001:000006dc       ??_C@_1BK@DDBMMJCN@?$AAW?$AAi?$AAd?$AAt?$AAh?$AAs?$AAR?$AAe?$AAm?$AAo?$AAt?$AAe?$AA?$AA@ 100016dc     Pclass.obj
 0001:000006f8       ??_C@_1BI@FOOHDOCI@?$AAW?$AAi?$AAd?$AAt?$AAh?$AAs?$AAL?$AAo?$AAc?$AAa?$AAl?$AA?$AA@ 100016f8     Pclass.obj
 0001:00000710       ??_C@_1BM@EDHFKJEJ@?$AAC?$AAo?$AAl?$AAu?$AAm?$AAn?$AAs?$AAR?$AAe?$AAm?$AAo?$AAt?$AAe?$AA?$AA@ 10001710     Pclass.obj
 0001:0000072c       ??_C@_1BK@HMOODHKK@?$AAC?$AAo?$AAl?$AAu?$AAm?$AAn?$AAs?$AAL?$AAo?$AAc?$AAa?$AAl?$AA?$AA@ 1000172c     Pclass.obj
 0001:00000748       ??_C@_1O@CBODAMOP@?$AAM?$AAo?$AAd?$AAe?$AA?$CF?$AAd?$AA?$AA@ 10001748     Pclass.obj
 0001:00000758       ??_C@_15LNKNCLHH@?$AAS?$AAs?$AA?$AA@ 10001758     Pclass.obj
 0001:00000760       ??_C@_13DEFPDAGF@?$AA?0?$AA?$AA@ 10001760     Pclass.obj
 0001:00000764       ??_C@_19MPDKCIDK@?$AA?5?$AA?$CF?$AAs?$AA?5?$AA?$AA@ 10001764     Pclass.obj
 0001:00000770       ??_C@_1BA@MFHNOFIJ@?$AA?$CF?$AAs?$AA?3?$AA?5?$AA?$CF?$AAs?$AA?5?$AA?$AA@ 10001770     Pclass.obj
 0001:00000780       ??_C@_13HOIJIPNN@?$AA?5?$AA?$AA@ 10001780     Pclass.obj
 0001:00000784       ??_C@_17JJIMNMHK@?$AA?5?$AA?$CG?$AA?$FO?$AA?$AA@ 10001784     Pclass.obj
 0001:0000078c       ??_C@_1M@EJMLOAMM@?$AA?$CF?$AA?9?$AA2?$AA2?$AAs?$AA?$AA@ 1000178c     Pclass.obj
 0001:00000798       ??_C@_17DJGLCLAO@?$AA?$CF?$AAs?$AA?3?$AA?$AA@ 10001798     Pclass.obj
 0001:000007a0       ??_C@_17JLFEDMMI@?$AA?$DP?$AA?$DP?$AA?$DP?$AA?$AA@ 100017a0     Pclass.obj
 0001:000007a8       ??_C@_1BO@EHJBCONC@?$AA?$CF?$AA0?$AA2?$AAd?$AA?3?$AA?$CF?$AA0?$AA2?$AAd?$AA?3?$AA?$CF?$AA0?$AA2?$AAd?$AA?$AA@ 100017a8     Pclass.obj
 0001:000007c8       ??_C@_1CE@OMPPCAIJ@?$AA?$CF?$AAd?$AA?5?$AA?$CF?$AA0?$AA2?$AAd?$AA?3?$AA?$CF?$AA0?$AA2?$AAd?$AA?3?$AA?$CF?$AA0?$AA2?$AAd?$AA?$AA@ 100017c8     Pclass.obj
 0001:0000081c       ??_C@_1CO@PDLCNLLF@?$AA?2?$AA?$CF?$AAs?$AA?2?$AA?$CF?$AAs?$AA?2?$AAF?$AAi?$AAl?$AAe?$AAD?$AAe?$AAs?$AAc?$AAr?$AAi?$AAp?$AAt?$AAi?$AAo?$AAn?$AA?$AA@ 1000181c     Pclass.obj
 0001:0000084c       ??_C@_1CG@PJJCHAJ@?$AA?2?$AA?$CF?$AAs?$AA?2?$AA?$CF?$AAs?$AA?2?$AAF?$AAi?$AAl?$AAe?$AAV?$AAe?$AAr?$AAs?$AAi?$AAo?$AAn?$AA?$AA@ 1000184c     Pclass.obj
 0001:00000894       ??_C@_19JHEHLFPM@?$AA?2?$AA?$DP?$AA?$DP?$AA?2?$AA?$AA@ 10001894     Pclass.obj
 0001:000008a0       ??_C@_1O@CIJHDDGA@?$AA?$CF?$AAs?$AA?5?$AA?$CF?$AAs?$AA?6?$AA?$AA@ 100018a0     Pclass.obj
 0001:000008b0       ??_C@_1O@DGEEABED@?$AA?$CF?$AAs?$AA?5?$AA?$CF?$AAd?$AA?6?$AA?$AA@ 100018b0     Pclass.obj
 0001:000008c0       ??_C@_1M@CBILFCKF@?$AA?5?$AA?$CI?$AA?$CF?$AAs?$AA?$CJ?$AA?$AA@ 100018c0     Pclass.obj
 0001:000008cc       ??_C@_17CHCGIDNB@?$AA?$CF?$AAs?$AA?2?$AA?$AA@ 100018cc     Pclass.obj
 0001:000008d4       ??_C@_17GMPJMPF@?$AA?$CF?$AAs?$AA?5?$AA?$AA@ 100018d4     Pclass.obj
 0001:000008dc       ??_C@_1BC@OMEIBLAI@?$AAw?$AAb?$AAe?$AAm?$AAc?$AAo?$AAm?$AAn?$AA?$AA@ 100018dc     Pclass.obj
 0001:000008f0       ??_7PluginEditFieldBinding@@6B@ 100018f0     Pclass.obj
 0001:000009b8       ??_C@_1CM@OLKFIHMK@?$AAN?$AA?0?$AAX?$AA1?$AA5?$AAT?$AA?0?$AAX?$AA1?$AA6?$AAT?$AA?0?$AAX?$AA1?$AA7?$AAT?$AA?0?$AAX?$AA1?$AA8?$AAS?$AA?$AA@ 100019b8     Pclass.obj
 0001:000009e4       ??_C@_1BG@MNPGDOEP@?$AA1?$AA2?$AA?0?$AA0?$AA?0?$AA0?$AA?0?$AA0?$AA?0?$AA4?$AA?$AA@ 100019e4     Pclass.obj
 0001:000009fc       ??_C@_1BO@ONCLJEFA@?$AAN?$AA?0?$AAX?$AAI?$AA?0?$AAX?$AAP?$AA?0?$AAX?$AA0?$AAS?$AA?0?$AAX?$AA6?$AA?$AA@ 100019fc     Pclass.obj
 0001:00000a1c       ??_C@_1BE@NCGLNDMK@?$AA0?$AA?0?$AA4?$AA?0?$AA2?$AA?0?$AA3?$AA?0?$AA9?$AA?$AA@ 10001a1c     Pclass.obj
 0001:00000a30       ??_C@_17KNGPBKAK@?$AAN?$AA?0?$AAN?$AA?$AA@ 10001a30     Pclass.obj
 0001:00000a38       ??_C@_17JPFFEOAH@?$AA0?$AA?0?$AA0?$AA?$AA@ 10001a38     Pclass.obj
 0001:00000a40       ??_C@_1BI@FAMBFJKE@?$AAN?$AA?0?$AAX?$AAI?$AA?0?$AAX?$AAC?$AA?0?$AAD?$AA?0?$AAT?$AA?$AA@ 10001a40     Pclass.obj
 0001:00000a58       ??_C@_1BE@MONBDOED@?$AA0?$AA?0?$AA4?$AA?0?$AA4?$AA?0?$AA0?$AA?0?$AA0?$AA?$AA@ 10001a58     Pclass.obj
 0001:00000a6c       ??_C@_1BG@MICALLFD@?$AAN?$AA?0?$AAX?$AAI?$AA?0?$AAX?$AA4?$AA?0?$AAX?$AA6?$AA?$AA@ 10001a6c     Pclass.obj
 0001:00000a84       ??_C@_1BA@CAEMMMKJ@?$AA0?$AA?0?$AA4?$AA?0?$AA9?$AA?0?$AA9?$AA?$AA@ 10001a84     Pclass.obj
 0001:00000a94       ??_C@_1DI@NKOPFHII@?$AAN?$AA?0?$AAX?$AAI?$AA?0?$AAX?$AA4?$AA?0?$AAX?$AA6?$AA?0?$AAX?$AA1?$AA0?$AA?0?$AAX?$AA1?$AA2?$AA?0?$AAX?$AA0?$AA?0?$AAX?$AA1?$AA?0?$AAX?$AA2?$AA?$AA@ 10001a94     Pclass.obj
 0001:00000acc       ??_C@_1CG@HGJJIJIH@?$AA1?$AA2?$AA?0?$AA4?$AA?0?$AA0?$AA?0?$AA0?$AA?0?$AA0?$AA?0?$AA0?$AA?0?$AA8?$AA?0?$AA8?$AA?0?$AA8?$AA?$AA@ 10001acc     Pclass.obj
 0001:00000af4       ??_C@_19ILLMDDHI@?$AAN?$AA?0?$AAZ?$AAD?$AA?$AA@ 10001af4     Pclass.obj
 0001:00000b00       ??_C@_19NMOJBHGD@?$AA1?$AA2?$AA?0?$AA0?$AA?$AA@ 10001b00     Pclass.obj
 0001:00000b10       ??_C@_1EA@HPDEOPPH@?$AAN?$AA?0?$AAX?$AAP?$AA?0?$AAX?$AA0?$AAS?$AA?0?$AAX?$AA1?$AAS?$AA?0?$AAX?$AA2?$AAS?$AA?0?$AAX?$AA1?$AA1?$AAS?$AA?0?$AAX?$AA1?$AA4?$AAS?$AA?0?$AAX?$AA1?$AA8?$AAS?$AA?$AA@ 10001b10     Pclass.obj
 0001:00000b50       ??_C@_1CA@MGMNHCLL@?$AA0?$AA?0?$AA2?$AA?0?$AA3?$AA?0?$AA2?$AA?0?$AA2?$AA?0?$AA3?$AA?0?$AA4?$AA?0?$AA3?$AA?$AA@ 10001b50     Pclass.obj
 0001:00000b70       ??_C@_1O@JGFFCAGM@?$AAN?$AA?0?$AAX?$AAI?$AA?0?$AAO?$AA?$AA@ 10001b70     Pclass.obj
 0001:00000b80       ??_C@_1O@LAHJLGAL@?$AA0?$AA?0?$AA5?$AA?0?$AA1?$AA5?$AA?$AA@ 10001b80     Pclass.obj
 0001:00000b90       ??_C@_1CC@FANCGEGE@?$AAN?$AA?0?$AAX?$AAI?$AA?0?$AAX?$AAT?$AA?0?$AAX?$AA3?$AA?0?$AAX?$AAG?$AA?0?$AAX?$AAU?$AA?$AA@ 10001b90     Pclass.obj
 0001:00000bb4       ??_C@_1BI@DGDJEDOL@?$AA0?$AA?0?$AA4?$AA?0?$AA3?$AA?0?$AA4?$AA?0?$AA4?$AA?0?$AA4?$AA?$AA@ 10001bb4     Pclass.obj
 0001:00000bcc       ??_C@_1BG@COBJEPBB@?$AAN?$AA?0?$AAX?$AAI?$AA?0?$AAX?$AAT?$AA?0?$AAX?$AA3?$AA?$AA@ 10001bcc     Pclass.obj
 0001:00000be4       ??_C@_1BA@EDOGAILM@?$AA0?$AA?0?$AA4?$AA?0?$AA3?$AA?0?$AA4?$AA?$AA@ 10001be4     Pclass.obj
 0001:00000bf4       ??_C@_15DNHPCDHG@?$AAT?$AAt?$AA?$AA@ 10001bf4     Pclass.obj
 0001:00000bfc       ??_C@_15JOGBDECP@?$AA?0?$AA?5?$AA?$AA@ 10001bfc     Pclass.obj
 0001:00000c04       ??_C@_1BE@PEGLKBKB@?$AA?6?$AA?$CF?$AAs?$AA?6?$AA?$CF?$AAs?$AA?$CF?$AAs?$AA?6?$AA?$AA@ 10001c04     Pclass.obj
 0001:00000c18       ??_C@_1BO@LJMHGFAK@?$AA?$CF?$AA?9?$AA2?$AA2?$AAs?$AA?5?$AA?$CF?$AA0?$AA8?$AAX?$AA?5?$AA?$CF?$AAs?$AA?6?$AA?$AA@ 10001c18     Pclass.obj
 0001:00000d58       ??_C@_1BE@JKDBKCGH@?$AA?$CF?$AA?9?$AA2?$AA2?$AAs?$AA?5?$AA?$CF?$AAp?$AA?6?$AA?$AA@ 10001d58     Pclass.obj
 0001:00000d6c       ??_C@_1M@NOMFOFMP@?$AAH?$AAW?$AAN?$AAD?$AA?3?$AA?$AA@ 10001d6c     Pclass.obj
 0001:00000d78       ??_C@_1BA@DHHNFIMD@?$AA?6?$AA?$CF?$AAs?$AA?5?$AA?$CF?$AAu?$AA?6?$AA?$AA@ 10001d78     Pclass.obj
 0001:00000d88       ??_C@_1BC@MLKIHIFN@?$AA?6?$AA?$CF?$AAs?$AA?3?$AA?6?$AA?$CF?$AAs?$AA?6?$AA?$AA@ 10001d88     Pclass.obj
 0001:00000d9c       ??_C@_1BG@MDLBKGIE@?$AA?6?$AA?$CF?$AAs?$AA?5?$AA?$CF?$AAs?$AA?5?$AA?$CF?$AAs?$AA?6?$AA?$AA@ 10001d9c     Pclass.obj
 0001:00000db4       ??_C@_1BA@OBCELLNO@?$AA?6?$AA?$CF?$AAs?$AA?5?$AA?$CF?$AAs?$AA?6?$AA?$AA@ 10001db4     Pclass.obj
 0001:00000dc4       ??_C@_1O@POMONAHN@?$AA?$CF?$AAs?$AA?5?$AA?$CF?$AAu?$AA?6?$AA?$AA@ 10001dc4     Pclass.obj
 0001:00000dd4       ??_C@_1M@LFADDFHG@?$AA?$CF?$AA0?$AA8?$AAX?$AA?6?$AA?$AA@ 10001dd4     Pclass.obj
 0001:00000de0       ??_C@_17BPBJDALC@?$AA?$CF?$AAu?$AA?6?$AA?$AA@ 10001de0     Pclass.obj
 0001:00000de8       ??_C@_1BE@OMBNFFBH@?$AA?$CF?$AAu?$AA?5?$AA?5?$AA?$CI?$AA?$CF?$AAs?$AA?$CJ?$AA?6?$AA?$AA@ 10001de8     Pclass.obj
 0001:00000dfc       ??_C@_1BC@CLLLJKLA@?$AA?$CF?$AAs?$AA?5?$AA?$CF?$AA0?$AA8?$AAX?$AA?6?$AA?$AA@ 10001dfc     Pclass.obj
 0001:00000e10       ??_C@_1BC@NEODPHBM@?$AA?$CF?$AAs?$AA?5?$AA?$CF?$AAs?$AA?$CF?$AAs?$AA?6?$AA?$AA@ 10001e10     Pclass.obj
 0001:00000e24       ??_C@_1O@CNKEJBH@?$AA?0?$AA?5?$AA?$CF?$AAd?$AA?$CF?$AAs?$AA?$AA@ 10001e24     Pclass.obj
 0001:00000e4c       ??_C@_19GGNHIDOH@?$AA?4?$AAt?$AAx?$AAt?$AA?$AA@ 10001e4c     Pclass.obj
 0001:00000e58       ??_C@_1BC@OMEIHGFC@?$AAW?$AAS?$AA_?$AAP?$AAO?$AAP?$AAU?$AAP?$AA?$AA@ 10001e58     Pclass.obj
 0001:00000e6c       ??_C@_1BC@ONEEOLLM@?$AAW?$AAS?$AA_?$AAC?$AAH?$AAI?$AAL?$AAD?$AA?$AA@ 10001e6c     Pclass.obj
 0001:00000e80       ??_C@_1BI@GHDIGAD@?$AAW?$AAS?$AA_?$AAM?$AAI?$AAN?$AAI?$AAM?$AAI?$AAZ?$AAE?$AA?$AA@ 10001e80     Pclass.obj
 0001:00000e98       ??_C@_1BG@KLPFHNBP@?$AAW?$AAS?$AA_?$AAV?$AAI?$AAS?$AAI?$AAB?$AAL?$AAE?$AA?$AA@ 10001e98     Pclass.obj
 0001:00000eb0       ??_C@_1BI@NKODCGOF@?$AAW?$AAS?$AA_?$AAD?$AAI?$AAS?$AAA?$AAB?$AAL?$AAE?$AAD?$AA?$AA@ 10001eb0     Pclass.obj
 0001:00000ec8       ??_C@_1CA@PCFJBBHH@?$AAW?$AAS?$AA_?$AAC?$AAL?$AAI?$AAP?$AAS?$AAI?$AAB?$AAL?$AAI?$AAN?$AAG?$AAS?$AA?$AA@ 10001ec8     Pclass.obj
 0001:00000ee8       ??_C@_1CA@MPLGGIO@?$AAW?$AAS?$AA_?$AAC?$AAL?$AAI?$AAP?$AAC?$AAH?$AAI?$AAL?$AAD?$AAR?$AAE?$AAN?$AA?$AA@ 10001ee8     Pclass.obj
 0001:00000f08       ??_C@_1BI@OLBAGOJG@?$AAW?$AAS?$AA_?$AAM?$AAA?$AAX?$AAI?$AAM?$AAI?$AAZ?$AAE?$AA?$AA@ 10001f08     Pclass.obj
 0001:00000f20       ??_C@_1BE@DAMMEKNP@?$AAW?$AAS?$AA_?$AAB?$AAO?$AAR?$AAD?$AAE?$AAR?$AA?$AA@ 10001f20     Pclass.obj
 0001:00000f34       ??_C@_1BI@EDHINADK@?$AAW?$AAS?$AA_?$AAD?$AAL?$AAG?$AAF?$AAR?$AAA?$AAM?$AAE?$AA?$AA@ 10001f34     Pclass.obj
 0001:00000f4c       ??_C@_1BG@CKCLFGFA@?$AAW?$AAS?$AA_?$AAV?$AAS?$AAC?$AAR?$AAO?$AAL?$AAL?$AA?$AA@ 10001f4c     Pclass.obj
 0001:00000f64       ??_C@_1BG@OMIOJOGF@?$AAW?$AAS?$AA_?$AAH?$AAS?$AAC?$AAR?$AAO?$AAL?$AAL?$AA?$AA@ 10001f64     Pclass.obj
 0001:00000f7c       ??_C@_1BG@KJOBMDJC@?$AAW?$AAS?$AA_?$AAS?$AAY?$AAS?$AAM?$AAE?$AAN?$AAU?$AA?$AA@ 10001f7c     Pclass.obj
 0001:00000f94       ??_C@_1BM@GPNNOPCH@?$AAW?$AAS?$AA_?$AAT?$AAH?$AAI?$AAC?$AAK?$AAF?$AAR?$AAA?$AAM?$AAE?$AA?$AA@ 10001f94     Pclass.obj
 0001:00000fb0       ??_C@_1BO@FODKBODI@?$AAW?$AAS?$AA_?$AAM?$AAI?$AAN?$AAI?$AAM?$AAI?$AAZ?$AAE?$AAB?$AAO?$AAX?$AA?$AA@ 10001fb0     Pclass.obj
 0001:00000fd0       ??_C@_1BO@IDJMAOMI@?$AAW?$AAS?$AA_?$AAM?$AAA?$AAX?$AAI?$AAM?$AAI?$AAZ?$AAE?$AAB?$AAO?$AAX?$AA?$AA@ 10001fd0     Pclass.obj
 0001:00000ff0       ??_C@_1CI@PKBCIOPN@?$AAW?$AAS?$AA_?$AAE?$AAX?$AA_?$AAD?$AAL?$AAG?$AAM?$AAO?$AAD?$AAA?$AAL?$AAF?$AAR?$AAA?$AAM?$AAE?$AA?$AA@ 10001ff0     Pclass.obj
 0001:00001018       ??_C@_1CK@KJECLHMG@?$AAW?$AAS?$AA_?$AAE?$AAX?$AA_?$AAN?$AAO?$AAP?$AAA?$AAR?$AAE?$AAN?$AAT?$AAN?$AAO?$AAT?$AAI?$AAF?$AAY?$AA?$AA@ 10002018     Pclass.obj
 0001:00001044       ??_C@_1BM@OCBKBALE@?$AAW?$AAS?$AA_?$AAE?$AAX?$AA_?$AAT?$AAO?$AAP?$AAM?$AAO?$AAS?$AAT?$AA?$AA@ 10002044     Pclass.obj
 0001:00001060       ??_C@_1CE@JIDMMICL@?$AAW?$AAS?$AA_?$AAE?$AAX?$AA_?$AAA?$AAC?$AAC?$AAE?$AAP?$AAT?$AAF?$AAI?$AAL?$AAE?$AAS?$AA?$AA@ 10002060     Pclass.obj
 0001:00001084       ??_C@_1CE@PFFPBMCF@?$AAW?$AAS?$AA_?$AAE?$AAX?$AA_?$AAT?$AAR?$AAA?$AAN?$AAS?$AAP?$AAA?$AAR?$AAE?$AAN?$AAT?$AA?$AA@ 10002084     Pclass.obj
 0001:000010a8       ??_C@_1BO@MEOEJPLO@?$AAW?$AAS?$AA_?$AAE?$AAX?$AA_?$AAM?$AAD?$AAI?$AAC?$AAH?$AAI?$AAL?$AAD?$AA?$AA@ 100020a8     Pclass.obj
 0001:000010c8       ??_C@_1CC@IEIGGJGG@?$AAW?$AAS?$AA_?$AAE?$AAX?$AA_?$AAT?$AAO?$AAO?$AAL?$AAW?$AAI?$AAN?$AAD?$AAO?$AAW?$AA?$AA@ 100020c8     Pclass.obj
 0001:000010ec       ??_C@_1CC@PLPNIKGL@?$AAW?$AAS?$AA_?$AAE?$AAX?$AA_?$AAW?$AAI?$AAN?$AAD?$AAO?$AAW?$AAE?$AAD?$AAG?$AAE?$AA?$AA@ 100020ec     Pclass.obj
 0001:00001110       ??_C@_1CC@IAPGCLEG@?$AAW?$AAS?$AA_?$AAE?$AAX?$AA_?$AAC?$AAL?$AAI?$AAE?$AAN?$AAT?$AAE?$AAD?$AAG?$AAE?$AA?$AA@ 10002110     Pclass.obj
 0001:00001134       ??_C@_1CE@EANKNCIF@?$AAW?$AAS?$AA_?$AAE?$AAX?$AA_?$AAC?$AAO?$AAN?$AAT?$AAE?$AAX?$AAT?$AAH?$AAE?$AAL?$AAP?$AA?$AA@ 10002134     Pclass.obj
 0001:00001158       ??_C@_1BI@GFIADCMK@?$AAW?$AAS?$AA_?$AAE?$AAX?$AA_?$AAR?$AAI?$AAG?$AAH?$AAT?$AA?$AA@ 10002158     Pclass.obj
 0001:00001170       ??_C@_1CC@JOFCJJPB@?$AAW?$AAS?$AA_?$AAE?$AAX?$AA_?$AAR?$AAT?$AAL?$AAR?$AAE?$AAA?$AAD?$AAI?$AAN?$AAG?$AA?$AA@ 10002170     Pclass.obj
 0001:00001194       ??_C@_1CI@EFLDECAB@?$AAW?$AAS?$AA_?$AAE?$AAX?$AA_?$AAL?$AAE?$AAF?$AAT?$AAS?$AAC?$AAR?$AAO?$AAL?$AAL?$AAB?$AAA?$AAR?$AA?$AA@ 10002194     Pclass.obj
 0001:000011bc       ??_C@_1CI@CIFGFFJB@?$AAW?$AAS?$AA_?$AAE?$AAX?$AA_?$AAC?$AAO?$AAN?$AAT?$AAR?$AAO?$AAL?$AAP?$AAA?$AAR?$AAE?$AAN?$AAT?$AA?$AA@ 100021bc     Pclass.obj
 0001:000011e4       ??_C@_1CC@BGEPLDCA@?$AAW?$AAS?$AA_?$AAE?$AAX?$AA_?$AAS?$AAT?$AAA?$AAT?$AAI?$AAC?$AAE?$AAD?$AAG?$AAE?$AA?$AA@ 100021e4     Pclass.obj
 0001:00001208       ??_C@_1CA@DOAIHHLO@?$AAW?$AAS?$AA_?$AAE?$AAX?$AA_?$AAA?$AAP?$AAP?$AAW?$AAI?$AAN?$AAD?$AAO?$AAW?$AA?$AA@ 10002208     Pclass.obj
 0001:00001228       ??_C@_1BM@FAODAMGD@?$AAW?$AAS?$AA_?$AAE?$AAX?$AA_?$AAL?$AAA?$AAY?$AAE?$AAR?$AAE?$AAD?$AA?$AA@ 10002228     Pclass.obj
 0001:00001244       ??_C@_1CM@DJKNBOGD@?$AAW?$AAS?$AA_?$AAE?$AAX?$AA_?$AAN?$AAO?$AAI?$AAN?$AAH?$AAE?$AAR?$AAI?$AAT?$AAL?$AAA?$AAY?$AAO?$AAU?$AAT?$AA?$AA@ 10002244     Pclass.obj
 0001:00001270       ??_C@_1CA@KMHLBMFI@?$AAW?$AAS?$AA_?$AAE?$AAX?$AA_?$AAL?$AAA?$AAY?$AAO?$AAU?$AAT?$AAR?$AAT?$AAL?$AA?$AA@ 10002270     Pclass.obj
 0001:00001290       ??_C@_1CC@LOFMDOPL@?$AAW?$AAS?$AA_?$AAE?$AAX?$AA_?$AAN?$AAO?$AAA?$AAC?$AAT?$AAI?$AAV?$AAA?$AAT?$AAE?$AA?$AA@ 10002290     Pclass.obj
 0001:000012b4       ??_C@_1BC@IALIJCAM@?$AAS?$AAo?$AAr?$AAt?$AAM?$AAo?$AAd?$AAe?$AA?$AA@ 100022b4     Pclass.obj
 0001:000012c8       ??_C@_1BO@OMKAPLPJ@?$AAS?$AAt?$AAa?$AAr?$AAt?$AAP?$AAa?$AAn?$AAe?$AAl?$AAM?$AAo?$AAd?$AAe?$AA?$AA@ 100022c8     Pclass.obj
 0001:000012e8       ??_C@_1M@MOFLFCEC@?$AA?$CF?$AAs?$AA?5?$AA?$CF?$AAs?$AA?$AA@ 100022e8     Pclass.obj
 0001:000012f4       ??_C@_1M@HKFBKEEN@?$AA?$CF?$AA?$CF?$AA?5?$AA?$CF?$AAs?$AA?$AA@ 100022f4     Pclass.obj
 0001:00001314       ??_C@_15LEKKCGMK@?$AA?2?$AA?2?$AA?$AA@ 10002314     Pclass.obj
 0001:0000131c       ??_C@_1CK@ECJCGOEK@?$AAP?$AAr?$AAo?$AAc?$AAe?$AAs?$AAs?$AAL?$AAi?$AAs?$AAt?$AA?4?$AAU?$AAs?$AAe?$AAr?$AAn?$AAa?$AAm?$AAe?$AA?$AA@ 1000231c     Pclass.obj
 0001:00001348       ??_C@_1CK@DGKCELDD@?$AAP?$AAr?$AAo?$AAc?$AAe?$AAs?$AAs?$AAL?$AAi?$AAs?$AAt?$AA?4?$AAC?$AAo?$AAm?$AAp?$AAu?$AAt?$AAe?$AAr?$AA?$AA@ 10002348     Pclass.obj
 0001:00001374       ??_C@_1BC@ENICKDH@?$AAC?$AAo?$AAn?$AAt?$AAe?$AAn?$AAt?$AAs?$AA?$AA@ 10002374     Pclass.obj
 0001:00001388       ??_C@_17FJPEEFCB@?$AAp?$AAr?$AAc?$AA?$AA@ 10002388     Pclass.obj
 0001:00001390       ??_C@_15DDHGOCBH@?$AA?4?$AA?4?$AA?$AA@ 10002390     Pclass.obj
 0001:00001398       ??_C@_1DA@BEHINMGJ@?$AAI?$AAO?$AA?5?$AAO?$AAt?$AAh?$AAe?$AAr?$AA?5?$AAO?$AAp?$AAe?$AAr?$AAa?$AAt?$AAi?$AAo?$AAn?$AAs?$AA?1?$AAs?$AAe?$AAc?$AA?$AA@ 10002398     perfthread.obj
 0001:000013c8       ??_C@_1DA@HICMAFKK@?$AAI?$AAO?$AA?5?$AAW?$AAr?$AAi?$AAt?$AAe?$AA?5?$AAO?$AAp?$AAe?$AAr?$AAa?$AAt?$AAi?$AAo?$AAn?$AAs?$AA?1?$AAs?$AAe?$AAc?$AA?$AA@ 100023c8     perfthread.obj
 0001:000013f8       ??_C@_1CO@LIIKBHDH@?$AAI?$AAO?$AA?5?$AAR?$AAe?$AAa?$AAd?$AA?5?$AAO?$AAp?$AAe?$AAr?$AAa?$AAt?$AAi?$AAo?$AAn?$AAs?$AA?1?$AAs?$AAe?$AAc?$AA?$AA@ 100023f8     perfthread.obj
 0001:00001428       ??_C@_1CO@LIEOHDCC@?$AAI?$AAO?$AA?5?$AAD?$AAa?$AAt?$AAa?$AA?5?$AAO?$AAp?$AAe?$AAr?$AAa?$AAt?$AAi?$AAo?$AAn?$AAs?$AA?1?$AAs?$AAe?$AAc?$AA?$AA@ 10002428     perfthread.obj
 0001:00001458       ??_C@_1CG@LBBBPCJA@?$AAI?$AAO?$AA?5?$AAO?$AAt?$AAh?$AAe?$AAr?$AA?5?$AAB?$AAy?$AAt?$AAe?$AAs?$AA?1?$AAs?$AAe?$AAc?$AA?$AA@ 10002458     perfthread.obj
 0001:00001480       ??_C@_1CG@MEJHKKKF@?$AAI?$AAO?$AA?5?$AAW?$AAr?$AAi?$AAt?$AAe?$AA?5?$AAB?$AAy?$AAt?$AAe?$AAs?$AA?1?$AAs?$AAe?$AAc?$AA?$AA@ 10002480     perfthread.obj
 0001:000014a8       ??_C@_1CE@EFLEKJAB@?$AAI?$AAO?$AA?5?$AAR?$AAe?$AAa?$AAd?$AA?5?$AAB?$AAy?$AAt?$AAe?$AAs?$AA?1?$AAs?$AAe?$AAc?$AA?$AA@ 100024a8     perfthread.obj
 0001:000014cc       ??_C@_1CE@DFDFLLAO@?$AAI?$AAO?$AA?5?$AAD?$AAa?$AAt?$AAa?$AA?5?$AAB?$AAy?$AAt?$AAe?$AAs?$AA?1?$AAs?$AAe?$AAc?$AA?$AA@ 100024cc     perfthread.obj
 0001:000014f0       ??_C@_1CG@KJOKFONA@?$AAV?$AAi?$AAr?$AAt?$AAu?$AAa?$AAl?$AA?5?$AAB?$AAy?$AAt?$AAe?$AAs?$AA?5?$AAP?$AAe?$AAa?$AAk?$AA?$AA@ 100024f0     perfthread.obj
 0001:00001518       ??_C@_1BM@FMIOMJAE@?$AAV?$AAi?$AAr?$AAt?$AAu?$AAa?$AAl?$AA?5?$AAB?$AAy?$AAt?$AAe?$AAs?$AA?$AA@ 10002518     perfthread.obj
 0001:00001534       ??_C@_1CA@GADAGCME@?$AAP?$AAa?$AAg?$AAe?$AA?5?$AAF?$AAa?$AAu?$AAl?$AAt?$AAs?$AA?1?$AAs?$AAe?$AAc?$AA?$AA@ 10002534     perfthread.obj
 0001:00001554       ??_C@_1BM@DGDPAMAA@?$AAP?$AAr?$AAi?$AAv?$AAa?$AAt?$AAe?$AA?5?$AAB?$AAy?$AAt?$AAe?$AAs?$AA?$AA@ 10002554     perfthread.obj
 0001:00001570       ??_C@_1CC@IMBAECJF@?$AAP?$AAo?$AAo?$AAl?$AA?5?$AAP?$AAa?$AAg?$AAe?$AAd?$AA?5?$AAB?$AAy?$AAt?$AAe?$AAs?$AA?$AA@ 10002570     perfthread.obj
 0001:00001594       ??_C@_1CI@LLKMGPEG@?$AAP?$AAo?$AAo?$AAl?$AA?5?$AAN?$AAo?$AAn?$AAp?$AAa?$AAg?$AAe?$AAd?$AA?5?$AAB?$AAy?$AAt?$AAe?$AAs?$AA?$AA@ 10002594     perfthread.obj
 0001:000015bc       ??_C@_1CC@OFJLEPCP@?$AAW?$AAo?$AAr?$AAk?$AAi?$AAn?$AAg?$AA?5?$AAS?$AAe?$AAt?$AA?5?$AAP?$AAe?$AAa?$AAk?$AA?$AA@ 100025bc     perfthread.obj
 0001:000015e0       ??_C@_1BI@GCOMDKEO@?$AAW?$AAo?$AAr?$AAk?$AAi?$AAn?$AAg?$AA?5?$AAS?$AAe?$AAt?$AA?$AA@ 100025e0     perfthread.obj
 0001:000015f8       ??_C@_1CK@FGGMBBIH@?$AAP?$AAa?$AAg?$AAe?$AA?5?$AAF?$AAi?$AAl?$AAe?$AA?5?$AAB?$AAy?$AAt?$AAe?$AAs?$AA?5?$AAP?$AAe?$AAa?$AAk?$AA?$AA@ 100025f8     perfthread.obj
 0001:00001624       ??_C@_1CA@KJMNGIDJ@?$AAP?$AAa?$AAg?$AAe?$AA?5?$AAF?$AAi?$AAl?$AAe?$AA?5?$AAB?$AAy?$AAt?$AAe?$AAs?$AA?$AA@ 10002624     perfthread.obj
 0001:00001644       ??_C@_1BK@FAAJNJIB@?$AAH?$AAa?$AAn?$AAd?$AAl?$AAe?$AA?5?$AAC?$AAo?$AAu?$AAn?$AAt?$AA?$AA@ 10002644     perfthread.obj
 0001:00001660       ??_C@_1BI@IIOPEKIO@?$AA?$CF?$AA?5?$AAU?$AAs?$AAe?$AAr?$AA?5?$AAT?$AAi?$AAm?$AAe?$AA?$AA@ 10002660     perfthread.obj
 0001:00001678       ??_C@_1CE@FNEMIHOD@?$AA?$CF?$AA?5?$AAP?$AAr?$AAi?$AAv?$AAi?$AAl?$AAe?$AAg?$AAe?$AAd?$AA?5?$AAT?$AAi?$AAm?$AAe?$AA?$AA@ 10002678     perfthread.obj
 0001:0000169c       ??_C@_1CC@DNHMJIKH@?$AA?$CF?$AA?5?$AAP?$AAr?$AAo?$AAc?$AAe?$AAs?$AAs?$AAo?$AAr?$AA?5?$AAT?$AAi?$AAm?$AAe?$AA?$AA@ 1000269c     perfthread.obj
 0001:000016c0       ??_C@_19DOGDICKI@?$AA?4?$AAe?$AAx?$AAe?$AA?$AA@ 100026c0     perfthread.obj
 0001:000016cc       ??_C@_19DLCFHDFF@?$AAP?$AAE?$AAR?$AAF?$AA?$AA@ 100026cc     perfthread.obj
 0001:000016d8       ??_C@_1BK@IKAFHKBD@?$AAE?$AAl?$AAa?$AAp?$AAs?$AAe?$AAd?$AA?5?$AAT?$AAi?$AAm?$AAe?$AA?$AA@ 100026d8     perfthread.obj
 0001:000016f4       ??_C@_1CI@FNIEMNAI@?$AAC?$AAr?$AAe?$AAa?$AAt?$AAi?$AAn?$AAg?$AA?5?$AAP?$AAr?$AAo?$AAc?$AAe?$AAs?$AAs?$AA?5?$AAI?$AAD?$AA?$AA@ 100026f4     perfthread.obj
 0001:0000171c       ??_C@_1BK@KCHPPKHP@?$AAT?$AAh?$AAr?$AAe?$AAa?$AAd?$AA?5?$AAC?$AAo?$AAu?$AAn?$AAt?$AA?$AA@ 1000271c     perfthread.obj
 0001:00001738       ??_C@_1BM@KCAKLHJN@?$AAP?$AAr?$AAi?$AAo?$AAr?$AAi?$AAt?$AAy?$AA?5?$AAB?$AAa?$AAs?$AAe?$AA?$AA@ 10002738     perfthread.obj
 0001:00001754       ??_C@_1BG@NKNJPBCD@?$AAI?$AAD?$AA?5?$AAP?$AAr?$AAo?$AAc?$AAe?$AAs?$AAs?$AA?$AA@ 10002754     perfthread.obj
 0001:0000176c       ??_C@_1BC@IICCDNLG@?$AAC?$AAo?$AAu?$AAn?$AAt?$AAe?$AAr?$AAs?$AA?$AA@ 1000276c     perfthread.obj
 0001:00001780       ??_C@_1HE@NBDABLAL@?$AAS?$AAo?$AAf?$AAt?$AAw?$AAa?$AAr?$AAe?$AA?2?$AAM?$AAi?$AAc?$AAr?$AAo?$AAs?$AAo?$AAf?$AAt?$AA?2?$AAW?$AAi?$AAn?$AAd?$AAo?$AAw?$AAs?$AA?5?$AAN?$AAT?$AA?2?$AAC?$AAu@ 10002780     perfthread.obj
 0001:000017f4       ??_C@_1CC@DMDJMJLM@?$AAS?$AAe?$AAD?$AAe?$AAb?$AAu?$AAg?$AAP?$AAr?$AAi?$AAv?$AAi?$AAl?$AAe?$AAg?$AAe?$AA?$AA@ 100027f4     Plist.obj
 0001:00001818       ??_C@_1M@GPDJLPMI@?$AA?4?$AA?$CF?$AA0?$AA3?$AAd?$AA?$AA@ 10002818     Plist.obj
 0001:00001824       ??_C@_1CC@EKFMKAAC@?$AA?$CF?$AA1?$AA0?$AA?4?$AA0?$AAf?$AA?5?$AA?5?$AA?$CF?$AA5?$AA?4?$AA0?$AAf?$AA?$CF?$AAs?$AA?6?$AA?$AA@ 10002824     Plist.obj
 0001:00001848       ??_C@_1BI@HAFBCFCK@?$AA?$CF?$AAs?$AA?5?$AA?$CF?$AA7?$AA?4?$AA0?$AAf?$AA?$CF?$AA?$CF?$AA?6?$AA?$AA@ 10002848     Plist.obj
 0001:00001860       ??_C@_1CG@FOOPEKLK@?$AA?$CF?$AA1?$AA0?$AAI?$AA6?$AA4?$AAu?$AA?5?$AA?5?$AA?$CF?$AA5?$AAI?$AA6?$AA4?$AAu?$AA?$CF?$AAs?$AA?6?$AA?$AA@ 10002860     Plist.obj
 0001:00001888       ??_C@_1BC@CIAMCHCM@?$AA?$CF?$AA1?$AA0?$AAI?$AA6?$AA4?$AAu?$AA?6?$AA?$AA@ 10002888     Plist.obj
 0001:0000189c       ??_C@_1BA@DJJLONDK@?$AA?$CF?$AA1?$AA0?$AA?4?$AA0?$AAf?$AA?6?$AA?$AA@ 1000289c     Plist.obj
 0001:000018ac       ??_C@_1O@KBBIJFEI@?$AA?$CF?$AA?9?$AA2?$AA4?$AAs?$AA?5?$AA?$AA@ 100028ac     Plist.obj
 0001:000018bc       ??_C@_13EBCNDICG@?$AA?3?$AA?$AA@ 100028bc     Plist.obj
 0001:000018c0       ??_C@_17MJEANDKP@?$AA?$CF?$AAs?$AA?6?$AA?$AA@ 100028c0     Plist.obj
 0001:000018c8       ??_C@_19FJPIAKGM@?$AA?$CF?$AAs?$AA?6?$AA?6?$AA?$AA@ 100028c8     Plist.obj
 0001:000018d4       ??_C@_1BA@LFJAMCEC@?$AA?$CF?$AAs?$AA?5?$AA?$CF?$AAs?$AA?6?$AA?6?$AA?$AA@ 100028d4     Plist.obj
 0001:000018e4       ??_C@_17ENEANJDH@?$AA?5?$AA?$CF?$AAs?$AA?$AA@ 100028e4     Plist.obj
 0001:000018ec       ??_C@_1BE@KPJOOIA@?$AA?5?$AA?5?$AA?$CF?$AAp?$AA?5?$AA?5?$AA?$CF?$AA6?$AAX?$AA?$AA@ 100028ec     Plist.obj
 0001:00001900       ??_C@_15JNBOKNOG@?$AA?$AN?$AA?6?$AA?$AA@ 10002900     Pmix.obj
 0001:00001908       ??_C@_1BG@FFJGBKCB@?$AAE?$AAr?$AAr?$AAo?$AAr?$AA?5?$AA0?$AAx?$AA?$CF?$AAx?$AA?$AA@ 10002908     Pmix.obj
 0001:00001920       _IID_IWbemLocator          10002920     WMI.obj
 0001:00001930       _CLSID_WbemLocator         10002930     WMI.obj
 0001:00001940       ??_C@_1DA@BIBEJFMF@?$AAW?$AAi?$AAn?$AA3?$AA2?$AA_?$AAP?$AAr?$AAo?$AAc?$AAe?$AAs?$AAs?$AA?4?$AAH?$AAa?$AAn?$AAd?$AAl?$AAe?$AA?$DN?$AA?$CF?$AAu?$AA?$AA@ 10002940     WMI.obj
 0001:00001970       ??_C@_1BO@CLCOBGDE@?$AAE?$AAx?$AAe?$AAc?$AAu?$AAt?$AAa?$AAb?$AAl?$AAe?$AAP?$AAa?$AAt?$AAh?$AA?$AA@ 10002970     WMI.obj
 0001:00001990       ??_C@_1BC@JHNNEHFE@?$AAP?$AAr?$AAi?$AAo?$AAr?$AAi?$AAt?$AAy?$AA?$AA@ 10002990     WMI.obj
 0001:000019a4       ??_C@_1O@OAMNPMOM@?$AAD?$AAo?$AAm?$AAa?$AAi?$AAn?$AA?$AA@ 100029a4     WMI.obj
 0001:000019b4       ??_C@_19PIJILKAI@?$AAU?$AAs?$AAe?$AAr?$AA?$AA@ 100029b4     WMI.obj
 0001:000019c0       ??_C@_1BC@HJJANEGO@?$AAG?$AAe?$AAt?$AAO?$AAw?$AAn?$AAe?$AAr?$AA?$AA@ 100029c0     WMI.obj
 0001:000019d4       ??_C@_17NKMLOKHF@?$AAS?$AAi?$AAd?$AA?$AA@ 100029d4     WMI.obj
 0001:000019dc       ??_C@_1BI@OIPNMPCL@?$AAG?$AAe?$AAt?$AAO?$AAw?$AAn?$AAe?$AAr?$AAS?$AAi?$AAd?$AA?$AA@ 100029dc     WMI.obj
 0001:000019f4       ??_C@_1BE@CFEJJKFE@?$AAS?$AAe?$AAs?$AAs?$AAi?$AAo?$AAn?$AAI?$AAd?$AA?$AA@ 100029f4     WMI.obj
 0001:00001a08       ??_C@_1BI@FLOHINJE@?$AAR?$AAe?$AAt?$AAu?$AAr?$AAn?$AAV?$AAa?$AAl?$AAu?$AAe?$AA?$AA@ 10002a08     WMI.obj
 0001:00001a20       ??_C@_1BM@MLGLIGHJ@?$AAW?$AAi?$AAn?$AA3?$AA2?$AA_?$AAP?$AAr?$AAo?$AAc?$AAe?$AAs?$AAs?$AA?$AA@ 10002a20     WMI.obj
 0001:00001a3c       ??_C@_1BI@NKNJJIDM@?$AAS?$AAe?$AAt?$AAP?$AAr?$AAi?$AAo?$AAr?$AAi?$AAt?$AAy?$AA?$AA@ 10002a3c     WMI.obj
 0001:00001a54       ??_C@_1BE@PBPGMODO@?$AAT?$AAe?$AAr?$AAm?$AAi?$AAn?$AAa?$AAt?$AAe?$AA?$AA@ 10002a54     WMI.obj
 0001:00001a68       ??_C@_1O@GGHBFGJC@?$AAR?$AAe?$AAa?$AAs?$AAo?$AAn?$AA?$AA@ 10002a68     WMI.obj
 0001:00001a78       ??_C@_1CA@ECJNGEII@?$AA?2?$AA?2?$AA?$CF?$AAs?$AA?2?$AAr?$AAo?$AAo?$AAt?$AA?2?$AAc?$AAi?$AAm?$AAv?$AA2?$AA?$AA@ 10002a78     WMI.obj
 0001:00001a98       ??_C@_13JOFGPIOO@?$AA?4?$AA?$AA@ 10002a98     WMI.obj
 0001:00001a9c       _MainGuid                  10002a9c     Proclist.obj
 0001:00001aac       _MenuGuid                  10002aac     Proclist.obj
 0001:00001abc       _ConfigDialogGuid          10002abc     Proclist.obj
 0001:00001acc       ??_C@_0BC@IOEGILCE@CoSetProxyBlanket?$AA@ 10002acc     Proclist.obj
 0001:00001ae0       ??_C@_1M@FFPAMFOB@?$AAo?$AAl?$AAe?$AA3?$AA2?$AA?$AA@ 10002ae0     Proclist.obj
 0001:00001aec       ??_C@_0BA@FKGDNIJG@GetGuiResources?$AA@ 10002aec     Proclist.obj
 0001:00001afc       ??_C@_1O@BCCLBEOE@?$AAu?$AAs?$AAe?$AAr?$AA3?$AA2?$AA?$AA@ 10002afc     Proclist.obj
 0001:00001b0c       ??_C@_0BD@MCBOPCDK@LookupAccountNameW?$AA@ 10002b0c     Proclist.obj
 0001:00001b20       ??_C@_0BD@LMGFHOAE@GetSidSubAuthority?$AA@ 10002b20     Proclist.obj
 0001:00001b34       ??_C@_0BI@LPFJALDI@GetSidSubAuthorityCount?$AA@ 10002b34     Proclist.obj
 0001:00001b4c       ??_C@_0BK@FIHGNING@GetSidIdentifierAuthority?$AA@ 10002b4c     Proclist.obj
 0001:00001b68       ??_C@_0L@KJHKJIPF@IsValidSid?$AA@ 10002b68     Proclist.obj
 0001:00001b74       ??_C@_1BC@DNHGCMLG@?$AAa?$AAd?$AAv?$AAa?$AAp?$AAi?$AA3?$AA2?$AA?$AA@ 10002b74     Proclist.obj
 0001:00001b88       ??_C@_0P@LKABJJMO@IsWow64Process?$AA@ 10002b88     Proclist.obj
 0001:00001b98       ??_C@_1BC@GDMECMAK@?$AAk?$AAe?$AAr?$AAn?$AAe?$AAl?$AA3?$AA2?$AA?$AA@ 10002b98     Proclist.obj
 0001:00001bac       ??_C@_0BH@DLPGICA@NtQueryInformationFile?$AA@ 10002bac     Proclist.obj
 0001:00001bc4       ??_C@_0BJ@NDLOPGCH@NtQuerySystemInformation?$AA@ 10002bc4     Proclist.obj
 0001:00001be0       ??_C@_0O@IFMDHOMC@NtQueryObject?$AA@ 10002be0     Proclist.obj
 0001:00001bf0       ??_C@_0BJ@HKKELGGC@NtQueryInformationThread?$AA@ 10002bf0     Proclist.obj
 0001:00001c0c       ??_C@_0BK@EGDDIFMK@NtQueryInformationProcess?$AA@ 10002c0c     Proclist.obj
 0001:00001c28       ??_C@_1M@OAIMIKLP@?$AAn?$AAt?$AAd?$AAl?$AAl?$AA?$AA@ 10002c28     Proclist.obj
 0001:00001c34       ??_C@_1DE@BGKMIKPD@?$AAE?$AAu?$AAg?$AAe?$AAn?$AAe?$AA?5?$AAR?$AAo?$AAs?$AAh?$AAa?$AAl?$AA?5?$AA?$CG?$AA?5?$AAF?$AAa?$AAr?$AA?5?$AAG?$AAr?$AAo?$AAu?$AAp?$AA?$AA@ 10002c34     Proclist.obj
 0001:00001c68       ??_C@_1DK@DCAMPEPJ@?$AAP?$AAr?$AAo?$AAc?$AAe?$AAs?$AAs?$AA?5?$AAL?$AAi?$AAs?$AAt?$AA?5?$AAf?$AAo?$AAr?$AA?5?$AAF?$AAA?$AAR?$AA?5?$AAM?$AAa?$AAn?$AAa?$AAg?$AAe?$AAr?$AA?$AA@ 10002c68     Proclist.obj
 0001:00001ca4       ??_C@_1BC@PDEABLIN@?$AAP?$AAr?$AAo?$AAc?$AAL?$AAi?$AAs?$AAt?$AA?$AA@ 10002ca4     Proclist.obj
 0001:00001cb8       ??_C@_1M@MNPEKPKO@?$AAp?$AAl?$AAi?$AAs?$AAt?$AA?$AA@ 10002cb8     Proclist.obj
 0001:00001cd0       __chkstk                   10002cd0 f   chkstk.obj
 0001:00001cd0       __alloca_probe             10002cd0     chkstk.obj
 0001:00001d00       ?fputc@@YAHHPAX@Z          10002d00 f   fileio.obj
 0001:00002600       ?PrintHandleInfo@@YA_NKPAX_NPAVPerfThread@@@Z 10003600 f   handles.obj
 0001:000027a0       ?GetLangString@PluginDialogBuilder@@MAEPB_WH@Z 100037a0 f i PCFG.OBJ
 0001:000027c0       ?Write@_Opt@@SAXXZ         100037c0 f   PCFG.OBJ
 0001:00002a10       ?Read@_Opt@@SAXXZ          10003a10 f   PCFG.OBJ
 0001:00002d40       ?SaveValue@?$DialogItemBinding@UFarDialogItem@@@@UAEXPAUFarDialogItem@@H@Z 10003d40 f i PCFG.OBJ
 0001:00002d40       ?InitDialogItem@?$DialogBuilderBase@UFarDialogItem@@@@MAEXPAUFarDialogItem@@PB_W@Z 10003d40 f i PCFG.OBJ
 0001:00002d50       ?TextWidth@?$DialogBuilderBase@UFarDialogItem@@@@MAEHABUFarDialogItem@@@Z 10003d50 f i PCFG.OBJ
 0001:00002d60       ?DoShowDialog@?$DialogBuilderBase@UFarDialogItem@@@@MAEHXZ 10003d60 f i PCFG.OBJ
 0001:00002d70       ??1?$DialogBuilderBase@UFarDialogItem@@@@MAE@XZ 10003d70 f i PCFG.OBJ
 0001:00002dc0       ??_G?$DialogBuilderBase@UFarDialogItem@@@@MAEPAXI@Z 10003dc0 f i PCFG.OBJ
 0001:00002dc0       ??_E?$DialogBuilderBase@UFarDialogItem@@@@MAEPAXI@Z 10003dc0 f i PCFG.OBJ
 0001:00002de0       ?ReallocDialogItems@?$DialogBuilderBase@UFarDialogItem@@@@IAEXXZ 10003de0 f i PCFG.OBJ
 0001:00002eb0       ?UpdateSecondColumnPosition@?$DialogBuilderBase@UFarDialogItem@@@@IAEXXZ 10003eb0 f i PCFG.OBJ
 0001:00002f10       ?SaveValues@?$DialogBuilderBase@UFarDialogItem@@@@IAEXXZ 10003f10 f i PCFG.OBJ
 0001:00002f60       ?MaxTextWidth@?$DialogBuilderBase@UFarDialogItem@@@@IAEHXZ 10003f60 f i PCFG.OBJ
 0001:00003020       ??1PluginDialogBuilder@@UAE@XZ 10004020 f i PCFG.OBJ
 0001:00003040       ?InitDialogItem@PluginDialogBuilder@@MAEXPAUFarDialogItem@@PB_W@Z 10004040 f i PCFG.OBJ
 0001:00003060       ?TextWidth@PluginDialogBuilder@@MAEHABUFarDialogItem@@@Z 10004060 f i PCFG.OBJ
 0001:00003080       ?DoShowDialog@PluginDialogBuilder@@MAEHXZ 10004080 f i PCFG.OBJ
 0001:000030e0       ??_G?$DialogItemBinding@UFarDialogItem@@@@UAEPAXI@Z 100040e0 f i PCFG.OBJ
 0001:000030e0       ??_GPluginCheckBoxBinding@@UAEPAXI@Z 100040e0 f i PCFG.OBJ
 0001:000030e0       ??_GPluginRadioButtonBinding@@UAEPAXI@Z 100040e0 f i PCFG.OBJ
 0001:000030e0       ??_GPluginIntEditFieldBinding@@UAEPAXI@Z 100040e0 f i PCFG.OBJ
 0001:000030e0       ??_EPluginEditFieldBinding@@UAEPAXI@Z 100040e0 f i Pclass.obj
 0001:000030e0       ??_EPluginCheckBoxBinding@@UAEPAXI@Z 100040e0 f i PCFG.OBJ
 0001:000030e0       ??_E?$DialogItemBinding@UFarDialogItem@@@@UAEPAXI@Z 100040e0 f i PCFG.OBJ
 0001:000030e0       ??_EPluginRadioButtonBinding@@UAEPAXI@Z 100040e0 f i PCFG.OBJ
 0001:000030e0       ??_EPluginIntEditFieldBinding@@UAEPAXI@Z 100040e0 f i PCFG.OBJ
 0001:000030e0       ??_GPluginEditFieldBinding@@UAEPAXI@Z 100040e0 f i Pclass.obj
 0001:00003100       ?SaveValue@PluginCheckBoxBinding@@UAEXPAUFarDialogItem@@H@Z 10004100 f i PCFG.OBJ
 0001:00003140       ?SaveValue@PluginRadioButtonBinding@@UAEXPAUFarDialogItem@@H@Z 10004140 f i PCFG.OBJ
 0001:00003170       ??0PluginIntEditFieldBinding@@QAE@ABUPluginStartupInfo@@PAPAXHPAHH@Z 10004170 f i PCFG.OBJ
 0001:00003210       ?SaveValue@PluginIntEditFieldBinding@@UAEXPAUFarDialogItem@@H@Z 10004210 f i PCFG.OBJ
 0001:00003240       ?CreateCheckBoxBinding@PluginDialogBuilder@@MAEPAU?$DialogItemBinding@UFarDialogItem@@@@PAHH@Z 10004240 f i PCFG.OBJ
 0001:00003290       ?CreateRadioButtonBinding@PluginDialogBuilder@@MAEPAU?$DialogItemBinding@UFarDialogItem@@@@PAH@Z 10004290 f i PCFG.OBJ
 0001:000032e0       ??_EPluginDialogBuilder@@UAEPAXI@Z 100042e0 f i PCFG.OBJ
 0001:000032e0       ??_GPluginDialogBuilder@@UAEPAXI@Z 100042e0 f i PCFG.OBJ
 0001:00003320       ?AddText@?$DialogBuilderBase@UFarDialogItem@@@@QAEPAUFarDialogItem@@H@Z 10004320 f i PCFG.OBJ
 0001:000033a0       ?AddCheckbox@?$DialogBuilderBase@UFarDialogItem@@@@QAEPAUFarDialogItem@@HPAHH_N@Z 100043a0 f i PCFG.OBJ
 0001:000034d0       ?AddSeparator@?$DialogBuilderBase@UFarDialogItem@@@@QAEXPB_W@Z 100044d0 f i PCFG.OBJ
 0001:00003540       ?UpdateBorderSize@?$DialogBuilderBase@UFarDialogItem@@@@IAEXXZ 10004540 f i PCFG.OBJ
 0001:000035c0       ??0PluginDialogBuilder@@QAE@ABUPluginStartupInfo@@ABU_GUID@@1HPB_WP6GHPAXHH3@Z3@Z 100045c0 f i PCFG.OBJ
 0001:000036c0       ?AddIntEditField@PluginDialogBuilder@@UAEPAUFarDialogItem@@PAHH@Z 100046c0 f i PCFG.OBJ
 0001:00003780       ?AddOKCancel@?$DialogBuilderBase@UFarDialogItem@@@@QAEXHHH_N@Z 10004780 f i PCFG.OBJ
 0001:000038f0       ?ShowDialog@?$DialogBuilderBase@UFarDialogItem@@@@QAE_NXZ 100048f0 f i PCFG.OBJ
 0001:00003930       ?Config@@YAHXZ             10004930 f   PCFG.OBJ
 0001:00003b30       ??0ui64Table@@QAE@XZ       10004b30 f   Pclass.obj
 0001:00003c20       ?SavePanelModes@Plist@@SAXXZ 10004c20 f   Pclass.obj
 0001:00003e70       ?TranslateMode@Plist@@CA_NPB_WPA_W@Z 10004e70 f   Pclass.obj
 0001:00004080       ?GeneratePanelModes@Plist@@AAEXXZ 10005080 f   Pclass.obj
 0001:00004630       ?PanelModes@Plist@@QAEPAUPanelMode@@AAI@Z 10005630 f   Pclass.obj
 0001:000046c0       ?GetOpenPanelInfo@Plist@@QAEXPAUOpenPanelInfo@@@Z 100056c0 f   Pclass.obj
 0001:000047c0       ?EnumWndProc@@YGHPAUHWND__@@J@Z 100057c0 f   Pclass.obj
 0001:00004840       ?FreeFindData@Plist@@QAEXPAUPluginPanelItem@@H@Z 10005840 f   Pclass.obj
 0001:000048a0       ?Reread@Plist@@AAEXXZ      100058a0 f   Pclass.obj
 0001:00004920       ?PutToCmdLine@Plist@@AAEXPA_W@Z 10005920 f   Pclass.obj
 0001:000049d0       ?PrintTitle@Plist@@SAPA_WH@Z 100059d0 f   Pclass.obj
 0001:00004a20       ?FileTimeToText@Plist@@AAEXPAU_FILETIME@@0PA_W@Z 10005a20 f   Pclass.obj
 0001:00004b40       ?GetVersionInfo@Plist@@SA_NPA_WAAPAEAAPA_W2@Z 10005b40 f   Pclass.obj
 0001:00004c90       ?PrintVersionInfo@Plist@@AAEXPAXPA_W@Z 10005c90 f   Pclass.obj
 0001:00004d60       ?ConnectWMI@Plist@@AAE_NXZ 10005d60 f   Pclass.obj
 0001:00004de0       ?PrintOwnerInfo@Plist@@AAEXPAXK@Z 10005de0 f   Pclass.obj
 0001:00004fd0       ?Compare@Plist@@QAEHPBUPluginPanelItem@@0I@Z 10005fd0 f   Pclass.obj
 0001:00005180       ?WmiError@Plist@@AAEXXZ    10006180 f   Pclass.obj
 0001:000051c0       ??0?$Array@_W@@QAE@K@Z     100061c0 f i Pclass.obj
 0001:00005200       ??0?$Array@UFarMenuItem@@@@QAE@K@Z 10006200 f i Pclass.obj
 0001:00005240       ?SaveValue@PluginEditFieldBinding@@UAEXPAUFarDialogItem@@H@Z 10006240 f i Pclass.obj
 0001:00005270       ?InitializePanelModes@Plist@@SAXXZ 10006270 f   Pclass.obj
 0001:000056c0       ?GetFindData@Plist@@QAEHAAPAUPluginPanelItem@@AAI_K@Z 100066c0 f   Pclass.obj
 0001:00005dd0       ?GetFiles@Plist@@QAEHPAUPluginPanelItem@@HHPAPB_W_KAAU_Opt@@@Z 10006dd0 f   Pclass.obj
 0001:00006b30       ?DeleteFiles@Plist@@QAEHPAUPluginPanelItem@@H_K@Z 10007b30 f   Pclass.obj
 0001:00006e10       ?ProcessEvent@Plist@@QAEHHPAX@Z 10007e10 f   Pclass.obj
 0001:00006fd0       ?DisconnectWMI@Plist@@AAEXXZ 10007fd0 f   Pclass.obj
 0001:00007000       ?EndColumns@?$DialogBuilderBase@UFarDialogItem@@@@QAEXXZ 10008000 f i Pclass.obj
 0001:000070c0       ?AddEditField@PluginDialogBuilder@@QAEPAUFarDialogItem@@PA_WHHPB_W_N@Z 100080c0 f i Pclass.obj
 0001:000071c0       ?AddPasswordField@PluginDialogBuilder@@QAEPAUFarDialogItem@@PA_WHH@Z 100081c0 f i Pclass.obj
 0001:00007290       ??0Plist@@QAE@XZ           10008290 f   Pclass.obj
 0001:00007410       ??1Plist@@QAE@XZ           10008410 f   Pclass.obj
 0001:00007460       ?Connect@Plist@@QAE_NPB_W00@Z 10008460 f   Pclass.obj
 0001:00007650       ?ProcessKey@Plist@@QAEHPBU_INPUT_RECORD@@@Z 10008650 f   Pclass.obj
 0001:00008590       ?SyncReread@PerfThread@@QAEXXZ 10009590 f   perfthread.obj
 0001:000085c0       ?GetProcessData@PerfThread@@QBEPAUProcessPerfData@@KK@Z 100095c0 f   perfthread.obj
 0001:00008620       ?Refresh@PerfThread@@AAEXXZ 10009620 f   perfthread.obj
 0001:00008ea0       ?RefreshWMIData@PerfThread@@AAEXXZ 10009ea0 f   perfthread.obj
 0001:00008fc0       ?ThreadProc@PerfThread@@AAGKXZ 10009fc0 f   perfthread.obj
 0001:00009080       ?ThreadProc@PerfThread@@CGKPAX@Z 1000a080 f   perfthread.obj
 0001:00009090       ??0PerfThread@@QAE@AAVPlist@@PB_W11@Z 1000a090 f   perfthread.obj
 0001:00009460       ??1PerfThread@@QAE@XZ      1000a460 f   perfthread.obj
 0001:000094e0       ?GetInternalProcessData@@YAHPAXPAU_LDR_MODULE@@AAPAU_RTL_USER_PROCESS_PARAMETERS@@AAPAD_N@Z 1000a4e0 f   Plist.obj
 0001:000095d0       ?GetPDataNT@@YA_NAAUProcessDataNT@@AAUProcessPerfData@@@Z 1000a5d0 f   Plist.obj
 0001:00009660       ?Enable@DebugToken@@QAE_NXZ 1000a660 f   Plist.obj
 0001:000096d0       ?Revert@DebugToken@@QAE_NXZ 1000a6d0 f   Plist.obj
 0001:00009710       ?CreateToken@DebugToken@@SA_NXZ 1000a710 f   Plist.obj
 0001:000097f0       ?CloseToken@DebugToken@@SAXXZ 1000a7f0 f   Plist.obj
 0001:00009810       ?PrintTime@@YAPA_WK_N@Z    1000a810 f   Plist.obj
 0001:000098a0       ?PrintTime@@YAPA_W_K_N@Z   1000a8a0 f   Plist.obj
 0001:00009910       ?DumpNTCounters@@YAXPAXAAVPerfThread@@KK@Z 1000a910 f   Plist.obj
 0001:00009bb0       ?PrintModuleVersion@@YAXPAXPA_W1H@Z 1000abb0 f   Plist.obj
 0001:00009c80       ?OpenProcessForced@@YAPAXPAVDebugToken@@KKH@Z 1000ac80 f   Plist.obj
 0001:00009cd0       ?GetList@@YAHAAPAUPluginPanelItem@@AAIAAVPerfThread@@@Z 1000acd0 f   Plist.obj
 0001:00009f80       ?GetOpenProcessData@@YAXPAXPA_WK1K1KPAPA_W2@Z 1000af80 f   Plist.obj
 0001:0000a260       ?KillProcess@@YAHKPAUHWND__@@@Z 1000b260 f   Plist.obj
 0001:0000a350       ?PrintNTCurDirAndEnv@@YAXPAX0H@Z 1000b350 f   Plist.obj
 0001:0000a490       ?PrintModules@@YAXPAXKAAU_Opt@@@Z 1000b490 f   Plist.obj
 0001:0000a6a0       ?GetMsg@@YAPB_WH@Z         1000b6a0 f   Pmix.obj
 0001:0000a6c0       ?ConvertDate@@YAXABU_FILETIME@@PA_W1@Z 1000b6c0 f   Pmix.obj
 0001:0000a750       ?WinError@@YAHPA_W@Z       1000b750 f   Pmix.obj
 0001:0000a8b0       ??0WMIConnection@@QAE@XZ   1000b8b0 f   WMI.obj
 0001:0000a8d0       ?GetProcessExecutablePath@WMIConnection@@QAEXKPA_W@Z 1000b8d0 f   WMI.obj
 0001:0000a9a0       ?GetProcessPriority@WMIConnection@@QAEKK@Z 1000b9a0 f   WMI.obj
 0001:0000aa60       ?GetProcessOwner@WMIConnection@@QAEXKPA_W0@Z 1000ba60 f   WMI.obj
 0001:0000abb0       ?GetProcessUserSid@WMIConnection@@QAEXKPA_W@Z 1000bbb0 f   WMI.obj
 0001:0000aca0       ?GetProcessSessionId@WMIConnection@@QAEHK@Z 1000bca0 f   WMI.obj
 0001:0000ad60       ?ExecMethod@WMIConnection@@AAEHKPB_W0K@Z 1000bd60 f   WMI.obj
 0001:0000af70       ?SetProcessPriority@WMIConnection@@QAEHKK@Z 1000bf70 f   WMI.obj
 0001:0000af90       ?TerminateProcess@WMIConnection@@QAEHK@Z 1000bf90 f   WMI.obj
 0001:0000afb0       ?Connect@WMIConnection@@QAE_NPB_W00@Z 1000bfb0 f   WMI.obj
 0001:0000b110       ?Disconnect@WMIConnection@@QAEXXZ 1000c110 f   WMI.obj
 0001:0000b130       ??1WMIConnection@@QAE@XZ   1000c130 f   WMI.obj
 0001:0000b160       __DllMainCRTStartup@12     1000c160 f   Proclist.obj
 0001:0000b1b0       ?AddIntEditField@?$DialogBuilderBase@UFarDialogItem@@@@UAEPAUFarDialogItem@@PAHH@Z 1000c1b0 f   PCFG.OBJ
 0001:0000b1b0       ?CreateCheckBoxBinding@?$DialogBuilderBase@UFarDialogItem@@@@MAEPAU?$DialogItemBinding@UFarDialogItem@@@@PAHH@Z 1000c1b0 f   PCFG.OBJ
 0001:0000b1c0       ?GetLangString@?$DialogBuilderBase@UFarDialogItem@@@@MAEPB_WH@Z 1000c1c0 f   PCFG.OBJ
 0001:0000b1c0       ?CreateRadioButtonBinding@?$DialogBuilderBase@UFarDialogItem@@@@MAEPAU?$DialogItemBinding@UFarDialogItem@@@@PAH@Z 1000c1c0 f   PCFG.OBJ
 0001:0000b340       ?Message@@YAHIPA_WPAPB_WHH@Z 1000c340 f   Proclist.obj
 0001:0000b370       _GetGlobalInfoW@4          1000c370 f   Proclist.obj
 0001:0000b3f0       _SetStartupInfoW@4         1000c3f0 f   Proclist.obj
 0001:0000b470       _ExitFARW@4                1000c470 f   Proclist.obj
 0001:0000b490       _ClosePanelW@4             1000c490 f   Proclist.obj
 0001:0000b4b0       _GetFindDataW@4            1000c4b0 f   Proclist.obj
 0001:0000b4d0       _FreeFindDataW@4           1000c4d0 f   Proclist.obj
 0001:0000b4f0       _GetPluginInfoW@4          1000c4f0 f   Proclist.obj
 0001:0000b5a0       _GetOpenPanelInfoW@4       1000c5a0 f   Proclist.obj
 0001:0000b5b0       _GetFilesW@4               1000c5b0 f   Proclist.obj
 0001:0000b5e0       _DeleteFilesW@4            1000c5e0 f   Proclist.obj
 0001:0000b600       _ProcessPanelEventW@4      1000c600 f   Proclist.obj
 0001:0000b620       _ProcessPanelInputW@4      1000c620 f   Proclist.obj
 0001:0000b640       _ConfigureW@4              1000c640 f   Proclist.obj
 0001:0000b650       _CompareW@4                1000c650 f   Proclist.obj
 0001:0000b670       _OpenW@4                   1000c670 f   Proclist.obj
 0001:0000b6f0       ??_V@YAXPAX@Z              1000c6f0 f   libCRT:delete_array.obj
 0001:0000b700       ??_U@YAPAXI@Z              1000c700 f   libCRT:new_array.obj
 0001:0000b710       __memicmp                  1000c710 f   libCRT:memicmp.obj
 0001:0000b780       _free                      1000c780 f   libCRT:free.obj
 0001:0000b7a0       _malloc                    1000c7a0 f   libCRT:malloc.obj
 0001:0000b7c0       ??3@YAXPAX@Z               1000c7c0 f   libCRT:delete.obj
 0001:0000b7d0       _memset                    1000c7d0 f   libCRT:memset.obj
 0001:0000b810       ??2@YAPAXI@Z               1000c810 f   libCRT:new.obj
 0001:0000b820       _wcschr                    1000c820 f   libCRT:strchr.obj
 0001:0000b850       _wcspbrk                   1000c850 f   libCRT:strpbrk.obj
 0001:0000b8a0       _wcsrchr                   1000c8a0 f   libCRT:strrchr.obj
 0001:0000b8d0       _wcstok                    1000c8d0 f   libCRT:strtok.obj
 0001:0000b990       _wcsdup                    1000c990 f   libCRT:strdup.obj
 0001:0000ba50       __ui64tow                  1000ca50 f   libCRT:i64toa.obj
 0001:0000ba80       __aulldiv                  1000ca80 f   libCRT:vc_ulldiv.obj
 0001:0000bc80       _wcstol                    1000cc80 f   libCRT:strtol.obj
 0001:0000bca0       _wcscspn                   1000cca0 f   libCRT:strcspn.obj
 0001:0000bcf0       _memcpy                    1000ccf0 f   libCRT:memcpy.obj
 0001:0000bd20       _wcsncat                   1000cd20 f   libCRT:strncat.obj
 0001:0000bd60       _memmove                   1000cd60 f   libCRT:memmove.obj
 0001:0000bdb0       __allmul                   1000cdb0 f   libCRT:vc_llmul.obj
 0001:0000bdf0       __alldiv                   1000cdf0 f   libCRT:vc_lldiv.obj
 0001:0000bea0       __aullrem                  1000cea0 f   libCRT:vc_ullrem.obj
 0001:0000bf20       __aulldvrm                 1000cf20 f   libCRT:vc_ulldvrm.obj
 0001:0000bfb6       _WNetCancelConnection2W@12 1000cfb6 f   mpr:MPR.dll
 0001:0000bfbc       _WNetAddConnection2W@16    1000cfbc f   mpr:MPR.dll
 0001:0000bfc2       _VerQueryValueW@16         1000cfc2 f   version:VERSION.dll
 0001:0000bfc8       _GetFileVersionInfoW@16    1000cfc8 f   version:VERSION.dll
 0001:0000bfce       _GetFileVersionInfoSizeW@8 1000cfce f   version:VERSION.dll
 0001:0000bfd4       __IMPORT_DESCRIPTOR_KERNEL32 1000cfd4     kernel32:KERNEL32.dll
 0001:0000bfe8       __IMPORT_DESCRIPTOR_USER32 1000cfe8     user32:USER32.dll
 0001:0000bffc       __IMPORT_DESCRIPTOR_ADVAPI32 1000cffc     advapi32:ADVAPI32.dll
 0001:0000c010       __IMPORT_DESCRIPTOR_ole32  1000d010     ole32:ole32.dll
 0001:0000c024       __IMPORT_DESCRIPTOR_MPR    1000d024     mpr:MPR.dll
 0001:0000c038       __IMPORT_DESCRIPTOR_VERSION 1000d038     version:VERSION.dll
 0001:0000c04c       __IMPORT_DESCRIPTOR_OLEAUT32 1000d04c     oleaut32:OLEAUT32.dll
 0001:0000c060       __NULL_IMPORT_DESCRIPTOR   1000d060     kernel32:KERNEL32.dll
 0002:00000000       ?DescIDs@@3PAHA            1000e000     Pclass.obj
 0002:00000080       ?Counters@@3PAU_Counters@@A 1000e080     perfthread.obj
 0002:00000188       ?pNtQueryInformationProcess@@3P6GJPAXW4_PROCESSINFOCLASS@@0KPAK@ZA 1000e188     Proclist.obj
 0002:0000018c       ?pNtQueryInformationThread@@3P6GJPAXK0KPAK@ZA 1000e18c     Proclist.obj
 0002:00000190       ?pNtQueryObject@@3P6GJPAXK0K0@ZA 1000e190     Proclist.obj
 0002:00000194       ?pNtQuerySystemInformation@@3P6GJKPAXKPAK@ZA 1000e194     Proclist.obj
 0002:00000198       ?pNtQueryInformationFile@@3P6GJPAX00KK@ZA 1000e198     Proclist.obj
 0002:0000019c       ?pIsWow64Process@@3P6GHPAXPAH@ZA 1000e19c     Proclist.obj
 0002:000001a0       ?pGetGuiResources@@3P6GKPAXK@ZA 1000e1a0     Proclist.obj
 0002:000001a4       ?pIsValidSid@@3P6GHPAX@ZA  1000e1a4     Proclist.obj
 0002:000001a8       ?pGetSidIdentifierAuthority@@3P6GPAU_SID_IDENTIFIER_AUTHORITY@@PAX@ZA 1000e1a8     Proclist.obj
 0002:000001ac       ?pGetSidSubAuthorityCount@@3P6GPAEPAX@ZA 1000e1ac     Proclist.obj
 0002:000001b0       ?pGetSidSubAuthority@@3P6GPAKPAXK@ZA 1000e1b0     Proclist.obj
 0002:000001b4       ?pLookupAccountName@@3P6GHPB_W0PAXPAKPA_W2PAW4_SID_NAME_USE@@@ZA 1000e1b4     Proclist.obj
 0002:000001b8       ?pCoSetProxyBlanket@@3P6GJPAUIUnknown@@KKPA_WKKPAXK@ZA 1000e1b8     Proclist.obj
 0002:000001c0       ?FPRINTFbuffer@@3PA_WA     1000e1c0     fileio.obj
 0002:000203c8       ?ProcPanelModesRemote@Plist@@2PAY0FA@_WA 1002e3c8     Pclass.obj
 0002:00020a08       ?PanelModesRemote@Plist@@2PAUPanelMode@@A 1002ea08     Pclass.obj
 0002:00020b48       ?bInit@Plist@@2_NA         1002eb48     Pclass.obj
 0002:00020b50       ?PanelModesLocal@Plist@@2PAUPanelMode@@A 1002eb50     Pclass.obj
 0002:00020c90       ?ProcPanelModesLocal@Plist@@2PAY0FA@_WA 1002ec90     Pclass.obj
 0002:000212d0       ?PanelModeBuffer@Plist@@2PA_WA 1002f2d0     Pclass.obj
 0002:00024fd0       __fltused                  10032fd0     Plist.obj
 0002:00024fd4       ?hDebugToken@DebugToken@@0RAXA 10032fd4     Plist.obj
 0002:00025028       ?Info@@3UPluginStartupInfo@@A 10033028     Proclist.obj
 0002:000250ac       ?_ui64Table@@3PAVui64Table@@A 100330ac     Proclist.obj
 0002:000250b0       ?PluginRootKey@@3PA_WA     100330b0     Proclist.obj
 0002:000250b4       ?Opt@@3U_Opt@@A            100330b4     Proclist.obj
 0002:000250d8       ?FSF@@3UFarStandardFunctions@@A 100330d8     Proclist.obj

 entry point at        0001:0000b160

 Static symbols

 0001:00001d30       ?GetProcessId@@YAHPAXAAK@Z 10002d30 f   handles.obj
 0001:00001d80       ?GetFileNameThread@@YGKPAX@Z 10002d80 f   handles.obj
 0001:00001dc0       ?PrintFileName@@YA_NPAX0@Z 10002dc0 f   handles.obj
 0001:00001ec0       ?GetTypeToken@@YA_NPAXPA_WK@Z 10002ec0 f   handles.obj
 0001:00001f40       ?GetTypeFromTypeToken@@YAGPB_W@Z 10002f40 f   handles.obj
 0001:00001f80       ?PrintNameByType@@YA_NPAXG0PAVPerfThread@@@Z 10002f80 f   handles.obj
 0001:00002280       ?PrintNameAndType@@YA_NPAXK0PAVPerfThread@@@Z 10003280 f   handles.obj
 0001:000023e0       ?ConvertSid@@YAHPAXPA_WPAK@Z 100033e0 f   handles.obj
 0001:00002510       ?GetUserAccountID@@YAPB_WXZ 10003510 f   handles.obj
 0001:00003b70       ?ui64toa_width@@YAX_KPA_WI_N@Z 10004b70 f   Pclass.obj
 0001:000042f0       ?GenerateTitles@@YAXQAY0FA@_WPAUPanelMode@@QAY0BI@PA_W@Z 100052f0 f   Pclass.obj
 0001:00008570       ?getcounter@@YAHPA_W@Z     10009570 f   perfthread.obj
 0001:00009650       ?FreeUserData@@YGXPAXPBUFarPanelItemFreeInfo@@@Z 1000a650 f   Plist.obj
 0001:0000b190       ?fNtQueryInformationProcess@@YGJPAXW4_PROCESSINFOCLASS@@0KPAK@Z 1000c190 f   Proclist.obj
 0001:0000b190       ?fNtQueryInformationThread@@YGJPAXK0KPAK@Z 1000c190 f   Proclist.obj
 0001:0000b190       ?fNtQueryObject@@YGJPAXK0K0@Z 1000c190 f   Proclist.obj
 0001:0000b190       ?fNtQueryInformationFile@@YGJPAX00KK@Z 1000c190 f   Proclist.obj
 0001:0000b1a0       ?fNtQuerySystemInformation@@YGJKPAXKPAK@Z 1000c1a0 f   Proclist.obj
 0001:0000b1b0       ?fGetGuiResources@@YGKPAXK@Z 1000c1b0 f   Proclist.obj
 0001:0000b1b0       ?fGetSidSubAuthority@@YGPAKPAXK@Z 1000c1b0 f   Proclist.obj
 0001:0000b1b0       ?fIsWow64Process@@YGHPAXPAH@Z 1000c1b0 f   Proclist.obj
 0001:0000b1c0       ?fGetSidSubAuthorityCount@@YGPAEPAX@Z 1000c1c0 f   Proclist.obj
 0001:0000b1c0       ?fGetSidIdentifierAuthority@@YGPAU_SID_IDENTIFIER_AUTHORITY@@PAX@Z 1000c1c0 f   Proclist.obj
 0001:0000b1c0       ?fIsValidSid@@YGHPAX@Z     1000c1c0 f   Proclist.obj
 0001:0000b1d0       ?fLookupAccountName@@YGHPB_W0PAXPAKPA_W2PAW4_SID_NAME_USE@@@Z 1000c1d0 f   Proclist.obj
 0001:0000b1e0       ?fCoSetProxyBlanket@@YGJPAUIUnknown@@KKPA_WKKPAXK@Z 1000c1e0 f   Proclist.obj
 0001:0000b1f0       ?dynamic_bind@@YAXXZ       1000c1f0 f   Proclist.obj
 0001:0000b9c0       ?x64toaw@@YAX_KPA_WIH@Z    1000c9c0 f   libCRT:i64toa.obj
 0001:0000baf0       ?strtoxl@@YAKPB_WPAPA_WHH@Z 1000caf0 f   libCRT:strtol.obj
